:10000000A2C20000D1C20000CFC20000CDC20000D9
:10001000CBC20000C9C20000C7C20000C5C20000B8
:10002000C3C20000C1C20000BFC20000BDC20000C8
:10003000BBC20000B9C20000B7C20000B5C20000D8
:10004000B3C200000C94CE09AFC20000ADC20000E4
:100050000C94FB09A9C20000A7C200000C947A0806
:10006000A3C200005AC600002FC600009DC20000B7
:100070009BC2000099C2000097C2000095C2000018
:100080000C94A10991C200008FC200008DC2000033
:100090008BC2000089C2000087C2000085C2000038
:1000A00083C2000081C200000C9474097DC200006C
:1000B0007BC2000079C2000077C200000C9447099F
:1000C00073C2000071C200006FC200006DC2000068
:1000D0006BC2000069C2000067C2000065C2000078
:1000E00063C2000012041504040408040E044C0446
:1000F00019041D04230427042B0431043504390496
:100100004C043F0443044704CC0AD30AD80ADD0A4E
:10011000E40AE90AD20CD20CD20CD20CD20CF00AAE
:10012000F70AFE0AD20C050B0A0B0F0B160B1B0B62
:10013000200B250B2A0B2F0BD20C340B390B3E0B4B
:10014000D20CD20CD20C430B480B4D0BD20CD20C60
:10015000520B590BD20CD20CD20C600B670B6E0BEE
:10016000D20C750B7A0B7F0BD20CD20CD20C840BF9
:10017000890B8E0BD20C950B9C0BA30BD20CD20CC3
:10018000D20CAA0BB10BB80BD20CBF0BC60BCD0B0C
:10019000D20CD20CD20CD40BDB0BE20BD20CD20C57
:1001A000D20CD20CD20CD20CD20CD20CD20CD20C5F
:1001B000D20CD20CD20CD20CD20CD20CD20CD20C4F
:1001C000D20CD20CD20CD20CD20CD20CD20CD20C3F
:1001D000D20CF80BFD0B020CD20C070C0C0C110C02
:1001E000D20CD20CD20C160C1D0C240CD20C2B0CE5
:1001F000320C390CD20CD20CD20C400C470C4E0CE9
:10020000D20C550C5A0C5F0CD20CD20CD20C640CD4
:10021000690C6E0CD20CD20CD20CD20CD20CD20CBB
:10022000D20CD20CD20CD20CD20CE90BEE0BF30B8D
:10023000D20CD20CD20CD20CD20CD20CD20CD20CCE
:10024000D20CD20CD20CD20CD20CD20CD20CD20CBE
:10025000D20CD20CD20CD20CD20CD20CD20CD20CAE
:10026000D20CD20CD20CD20CD20CD20CD20CD20C9E
:10027000D20CD20CD20CD20CD20CD20CD20CD20C8E
:10028000D20CD20CD20CD20CD20CD20CD20CD20C7E
:10029000D20CD20CD20CD20CD20C730C780C7F0C7A
:1002A000D20C860C8B0C920CD20CD20CD20C990C6A
:1002B0009E0CA50CD20CAC0CB10CB80CD20CD20C10
:1002C000D20CBF0CC40CCB0C921597159C15A6151F
:1002D000B0152916BA15C215CA15D415DE15E815BC
:1002E000F715011629160B1615161F1600000A0B16
:1002F00002090C0D0E0807030401000000000000B5
:1003000000000000000000000000000000000000ED
:1003100000000000000000001211100000000000AA
:1003200000000000000000000000000000000000CD
:10033000000000002100240027002A002D003000CA
:10034000330001010000040107010A01000022003E
:10035000250028002B002E0031003400020100008F
:10036000050108010B0100002000230026002900E0
:100370002C002F00320000010000030106010901DA
:1003800005050505070508080808020202020A0A11
:10039000080804040404010101010101010103032F
:1003A000030303030303040707070C0C0C0C0C0CDA
:1003B0000C0C0202020206060606060606060B0BD7
:1003C0000B0B0B0B0B0B0102102020080810204018
:1003D0001020408002010201080402010102040809
:1003E0001020408080402010080402018004020197
:1003F00080402010080402010804020101020408E0
:100400001020408001020408102040804E414E49D7
:100410004E495459494E46CDCCCC3D0AD7233C17C2
:10042000B7D13877CC2B329595E6241FB14F0A000F
:100430000020410000C84200401C4620BCBE4CCAFF
:100440001B0E5AAEC59D7400407A10F35A00A0727C
:100450004E18090010A5D4E80000E87648170000FF
:10046000E40B54020000CA9A3B000000E1F50500CD
:100470000080969800000040420F000000A0860116
:10048000000000102700000000E8030000000064E6
:1004900000000000000A0000000000010000000051
:1004A000002C76D888DC674F0823DFC1DFAE59E126
:1004B000B1B796E5E3E453C63AE651997696E8E695
:1004C000C28426EB898C9B62ED407C6FFCEFBC9C68
:1004D0009F40F2BAA56FA5F490055A2AF75C936B7A
:1004E0006CF9676DC11BFCE0E40D47FEF520E6B535
:1004F00000D0ED902E0300943577050080841E080F
:100500000000204E0A000000C80C333333330F982C
:100510006E12831141EF8D2114893BE65516CFFEF3
:10052000E6DB18D1844B381BF77C1D901DA4BBE47F
:1005300024203284725E228100C9F124ECA1E53DC1
:10054000270064415F4111241FBECFEFD1E2DEBF1F
:10055000CDBF00E00CBF17E0A0E0B2E0E2EEF6E9AC
:1005600000E00BBF02C007900D92A635B107D9F786
:100570002BE0A6E5B7E001C01D92A834B207E1F771
:1005800012E0C2EAD2E000E006C021970109802F04
:10059000FE010E94EB41C13AD10780E00807A9F7AC
:1005A0000E941B380C945F4B2BCDCF92DF92EF92C1
:1005B000FF920F931F93CF93DF936C017A018B010E
:1005C000C0E0D0E0CE15DF0589F0D8016D918D0136
:1005D000D601ED91FC910190F081E02DC6011995B5
:1005E000892B11F47E0102C02196ECCFC701DF9167
:1005F000CF911F910F91FF90EF90DF90CF900895D2
:10060000FC01918D828D981761F0828DDF01A80F1A
:10061000B11D5D968C91928D9F5F9F73928F90E03C
:1006200008958FEF9FEF0895FC01918D828D9817AB
:1006300031F0828DE80FF11D858D90E008958FEFE8
:100640009FEF0895FC01918D228D892F90E0805CB1
:100650009F4F821B91098F739927089584E09AE038
:10066000F1DF21E0892B09F420E0822F0895FC01BD
:10067000848DDF01A80FB11DA35ABF4F2C91848D2B
:1006800090E001968F739927848FA689B7892C9360
:10069000A089B1898C9180648C93938D848D9813FB
:1006A00006C00288F389E02D80818F7D80830895C4
:1006B000EF92FF920F931F93CF93DF93EC0181E0B2
:1006C000888F9B8D8C8D981305C0E889F98980816E
:1006D00085FD23C0F62E0B8D10E00F5F1F4F0F73AB
:1006E0001127E02E8C8DE8120BC00FB607FCFACF55
:1006F000E889F989808185FFF5CFCE01B8DFF2CF97
:100700008B8DFE01E80FF11DE35AFF4FF0820B8F36
:10071000EA89FB898081806207C0EE89FF89608356
:10072000E889F98980818064808381E090E0DF91AD
:10073000CF911F910F91FF90EF900895CF93DF938A
:10074000EC01888D8823C1F0EA89FB89808185FDD1
:1007500005C0A889B9898C9186FD0EC00FB607FC2B
:10076000F5CF808185FFF2CFA889B9898C9185FF6B
:10077000EDCFCE017CDFE8CFDF91CF91089580E00F
:1007800090E0892B19F06ADF811125C080E090E0AC
:10079000892B41F080E090E0892B21F00E9400003D
:1007A00081111CC080E090E0892B41F080E090E056
:1007B000892B21F00E940000811113C080E090E09D
:1007C000892BA1F080E090E0892B81F00E9400004D
:1007D00081110AC008950E940000D8CF0E94000035
:1007E000E1CF0E940000EACF0C940000089590E051
:1007F000FC013197E231F10508F04EC08827EE5830
:10080000FF4F8F4F0C94EB41809180008F7703C096
:10081000809180008F7D809380000895809180007A
:10082000877FF9CF84B58F7702C084B58F7D84BD73
:1008300008958091B0008F7703C08091B0008F7DC4
:100840008093B0000895809190008F7707C08091C9
:1008500090008F7D03C080919000877F80939000EF
:1008600008958091A0008F7707C08091A0008F7DB0
:1008700003C08091A000877F8093A000089580919D
:1008800020018F7707C0809120018F7D03C0809168
:100890002001877F8093200108953FB7F8948091CD
:1008A000EC099091ED09A091EE09B091EF0926B500
:1008B000A89B05C02F3F19F00196A11DB11D3FBF98
:1008C000BA2FA92F982F8827820F911DA11DB11D26
:1008D000BC01CD0142E0660F771F881F991F4A9522
:1008E000D1F708950F93FC019285908783858187C6
:1008F000A689B789119721F4621721F0401711F0EA
:100900006287438783858823D1F0828591110AC04D
:100910008823A9F080899189A289B3890197A109C7
:10092000B10909C081110BC080899189A289B3895D
:100930000196A11DB11D808B918BA28BB38B0F9162
:100940000895EBE0F1E08081877F80830895EBE0FC
:10095000F1E080818860808308958E9808958E9A52
:10096000089514980895149A089588980895889A77
:1009700008950E94ED430F931F93CF93DF93EC01F3
:1009800088819981009729F02A813B8126173707B2
:1009900088F48B016F5F7F4F0E940943009761F0DD
:1009A000998388831B830A832C813D81232B11F437
:1009B000FC01108281E001C080E0DF91CF911F91A6
:1009C0000F9108950F931F93CF93DF938091E109C7
:1009D0009091E20901969093E2098093E109809158
:1009E000E0098111BDC059DF6093DC097093DD0916
:1009F0008093DE099093DF0981E08093E0090E94F3
:100A00006D14EC0106B126B1409100016091000126
:100A10000295017026FB222720F9417066956170CE
:100A200085589E4F5FDF06B126B140B160B10170BD
:100A300022FB222720F943FB442740F96695617089
:100A4000CE018B569E4F4EDF02B322B340B160B150
:100A5000017022FB222720F9441F4427441F65FB15
:100A6000662760F9CE0181559E4F3CDFFE01E259B9
:100A7000FF4F8081882361F0709780819181A281EE
:100A8000B3810196A11DB11D80839183A283B3839D
:100A9000FE01E951FF4F8081882361F070978081CA
:100AA0009181A281B3810196A11DB11D80839183A3
:100AB000A283B383FE01E05AFE4F8081882369F050
:100AC000C05BDE4F88819981AA81BB810196A11DFF
:100AD000B11D88839983AA83BB83DFDE6093D80925
:100AE0007093D9098093DA099093DB090091DC09AE
:100AF0001091DD092091DE093091DF0906171707F3
:100B00002807390770F4DC01CB01801B910BA20B85
:100B1000B30B8093D4099093D509A093D609B093D1
:100B2000D7098091D4099091D509A091D609B091A7
:100B3000D7094091D0095091D1096091D2097091A3
:100B4000D309481759076A077B0740F48093D009F7
:100B50009093D109A093D209B093D3091092E009E0
:100B6000DF91CF911F910F910895EF92FF920F9314
:100B70001F93CF93DF93FC012481358161157105AB
:100B800011F480E018C041155105A1F07B01EC0182
:100B90008A01020F131FB801EEDE882391F328812A
:100BA00039818C819D81B701820F931F0E9403447C
:100BB0001D830C8381E0DF91CF911F910F91FF90F6
:100BC000EF900895EF92FF920F931F93CF93DF93CF
:100BD000CDB7DEB764970FB6F894DEBF0FBECDBFBA
:100BE0007C01CB01BA018E010F5F1F4F22E044E070
:100BF0000E940A44BC01FC0101900020E9F73197F2
:100C0000AF01481B590BC701B0DF64960FB6F894CB
:100C1000DEBF0FBECDBFDF91CF911F910F91FF902F
:100C2000EF9008956115710549F0FB0101900020D6
:100C3000E9F73197AF01461B570B97CF80E0089536
:100C4000FB0144815581608171818FCFEF92FF92CA
:100C50000F931F93CF93DF93EC017B018A01BA01BD
:100C60008ADE2881398181110DC02115310519F0E5
:100C7000C9010E94BE44198218821D821C821B82F7
:100C80001A8206C01D830C83B701C9010E94034468
:100C9000CE01DF91CF911F910F91FF90EF900895BA
:100CA000FC01118210821382128215821482611556
:100CB000710549F0FB0101900020E9F73197AF0180
:100CC000461B570BC3CF08951F920F920FB60F927A
:100CD00011240BB60F922F933F934F935F936F9313
:100CE0007F938F939F93AF93BF93EF93FF9384E092
:100CF0009AE0BDDCFF91EF91BF91AF919F918F91F1
:100D00007F916F915F914F913F912F910F900BBE0B
:100D10000F900FBE0F901F9018951F920F920FB655
:100D20000F9211240BB60F922F938F939F93EF93F3
:100D3000FF93E091140AF091150A8081E0911A0A5C
:100D4000F0911B0A82FD12C0908180911D0A8F5F75
:100D50008F7320911E0A821751F0E0911D0AF0E076
:100D6000EC5FF54F958F80931D0A01C08081FF9144
:100D7000EF919F918F912F910F900BBE0F900FBE0F
:100D80000F901F901895CF93DF93282F30E0F90133
:100D9000E451FD4F8491F901EA53FC4FD491F901DC
:100DA000E058FC4FC491CC2389F0811120DDEC2F59
:100DB000F0E0EE0FFF1FEA59FC4FA591B491EC91C2
:100DC000ED2381E090E021F480E002C080E090E03B
:100DD000DF91CF9108951F93CF93DF93282F30E0B9
:100DE000F901E451FD4F8491F901EA53FC4FD4918C
:100DF000F901E058FC4FC491CC23C1F0162F8111AA
:100E0000F6DCEC2FF0E0EE0FFF1FE45BFC4FA5914A
:100E1000B4918FB7F894111105C09C91ED2FE09516
:100E2000E92302C0EC91ED2BEC938FBFDF91CF91C2
:100E30001F910895CF92DF92EF92FF920F931F932D
:100E4000CF93DF936C018B017A01EC01CD51D64F2A
:100E5000888187FF04C0FB011182108224C08CE0CE
:100E60008C9D90018D9D300D11248881A901480F22
:100E7000511D87FD5A958091390B90E0481759070D
:100E800094F48881A901480F511D87FD5A95CA0124
:100E9000FA01EE0FFF1F8E0F9F1FFC01E755F54F64
:100EA000808186FD19C088818F5F88838CE08C9D4E
:100EB00090018D9D300D11248881A901480F511D8D
:100EC00087FD5A958091390B90E048175907B4F483
:100ED00088818C303CF112C08881280F311D87FD3C
:100EE0003A95F901EE0FFF1F2E0F3F1FF901E7554D
:100EF000F54F808160E08F736EDFD5CFF801808180
:100F00009181049680349C4918F480E49CE904C0E3
:100F1000F801808191810496F701918380838FEF9E
:100F2000888344C0F801408151818881B901680FEC
:100F3000711D87FD7A95CB01FB01EE0FFF1F8E0F10
:100F40009F1FFC01E755F54F81819281840F951F0A
:100F5000F701918380838881A901480F511D87FD86
:100F60005A95CA01FA01EE0FFF1F8E0F9F1FFC0159
:100F7000E755F54F808186FF19C08881280F311D04
:100F800087FD3A95F901EE0FFF1F2E0F3F1FF90164
:100F9000E755F54F808161E08F73DF91CF911F910D
:100FA0000F91FF90EF90DF90CF9015CFDF91CF9111
:100FB0001F910F91FF90EF90DF90CF90089560E028
:100FC000FC01838508CF60E0FC01858104CF61E0EE
:100FD000FC01838500CF61E0FC018581FCCECF93CD
:100FE000DF9390E0FC01EA53FC4F2491FC01E058B0
:100FF000FC4F8491882361F190E0880F991FFC01D8
:10100000EE5CFC4FC591D491FC01E45BFC4FA591D3
:10101000B491611109C09FB7F8948881209582230B
:101020008883EC912E230BC0623061F49FB7F89453
:101030003881822F809583238883EC912E2B2C93EB
:101040009FBF06C08FB7F894E8812E2B28838FBFEF
:10105000DF91CF9108958230910538F0880F991F64
:10106000880F991F05970197F1F708958F929F9226
:10107000AF92BF92CF92DF92EF92FF926B017C0111
:101080000CDC4B015C01C114D104E104F104E9F072
:1010900004DCDC01CB0188199909AA09BB09883E47
:1010A0009340A105B10578F321E0C21AD108E10807
:1010B000F10888EE880E83E0981EA11CB11CC114B3
:1010C000D104E104F10421F7DECFFF90EF90DF902F
:1010D000CF90BF90AF909F908F9008952FB7F894C6
:1010E0006091E8097091E9098091EA099091EB0912
:1010F0002FBF08951F920F920FB60F9211242F93B6
:101100003F938F939F93AF93BF938091E809909102
:10111000E909A091EA09B091EB093091E70923E0D0
:10112000230F2D3720F40196A11DB11D05C026E81F
:10113000230F0296A11DB11D2093E7098093E809B2
:101140009093E909A093EA09B093EB098091EC0927
:101150009091ED09A091EE09B091EF090196A11DC2
:10116000B11D8093EC099093ED09A093EE09B09323
:10117000EF09BF91AF919F918F913F912F910F9068
:101180000FBE0F901F901895CF92DF92EF92FF92B3
:10119000CF93DF93EC01603282E078070CF03DC022
:1011A00077FD06C0653B71052CF064EB70E002C072
:1011B00060E070E0898128E830E06901C81AD10850
:1011C00087FDD394CC0CDD1CCC0CDD1C0D2C000C4D
:1011D000EE08FF088A8128E532E0281B310987FDE7
:1011E0003395220F331F220F331FC901330FAA0B70
:1011F000BB0B9C01AD012C193D094E095F09DB01B8
:101200000E94284B24EB30E040E050E00E94024B6B
:10121000C20ED31EE41EF51EB6018881803380F510
:10122000998148E850E0491B510997FD5395440FB7
:10123000551F440F551F6417750784F09A8128E5E0
:1012400032E0291B310997FD3395220F331F220FFE
:10125000331FAB01261737070CF4A901425051097F
:10126000440F551F2FB7F89490E0FC01EE0FFF1FBD
:101270008E0F9F1FFC01E755F54F528341832FBF0F
:10128000DF91CF91FF90EF90DF90CF9008951F9264
:101290000F920FB60F9211240BB60F922F933F931C
:1012A0004F935F936F937F938F939F93AF93BF936E
:1012B000EF93FF9348E251E064E271E080E090E058
:1012C000B9DDFF91EF91BF91AF919F918F917F9188
:1012D0006F915F914F913F912F910F900BBE0F90A7
:1012E0000FBE0F901F9018951F920F920FB60F927E
:1012F00011240BB60F922F933F934F935F936F93ED
:101300007F938F939F93AF93BF93EF93FF9348EA9D
:1013100050E064EA70E083E090E08CDDFF91EF91B3
:10132000BF91AF919F918F917F916F915F914F91FD
:101330003F912F910F900BBE0F900FBE0F901F90FB
:1013400018951F920F920FB60F9211240BB60F92A1
:101350002F933F934F935F936F937F938F939F93BD
:10136000AF93BF93EF93FF9348E950E064E970E0D7
:1013700082E090E05FDDFF91EF91BF91AF919F918F
:101380008F917F916F915F914F913F912F910F902E
:101390000BBE0F900FBE0F901F9018951F920F92CB
:1013A0000FB60F9211240BB60F922F933F934F93CA
:1013B0005F936F937F938F939F93AF93BF93EF93BD
:1013C000FF9348E850E064E870E081E090E032DDAF
:1013D000FF91EF91BF91AF919F918F917F916F910D
:1013E0005F914F913F912F910F900BBE0F900FBEC9
:1013F0000F901F9018951F920F920FB60F92112405
:101400000BB60F922F933F934F935F936F937F93FE
:101410008F939F93AF93BF93EF93FF93E091560702
:10142000F09157071995FF91EF91BF91AF919F915F
:101430008F917F916F915F914F913F912F910F907D
:101440000BBE0F900FBE0F901F901895CF93DF9398
:10145000EC01888198DC21E0892B09F420E02C87BD
:101460008C8191DC21E0892B09F420E02E878E8984
:101470009F890197C1F48A8186DC21E0892B09F4D8
:1014800020E02D878E817FDC21E0892B09F420E08C
:101490002F879C858D85981749F08E85821731F0AE
:1014A0009A878B8703C08C858A872B87DF91CF91A2
:1014B0000895CF93DF93FC01A489B589C08DD18DA8
:1014C0002089318942895389A436B10559F01A1609
:1014D0001B0644F40E94284B24E630E040E050E034
:1014E0000E94024BDE010E94284BDF91CF910895AC
:1014F000FC011182108215821482108A118A128ACC
:10150000138A178A168A84E690E0958B848B12865C
:10151000108614861586168617860895CF93DF9356
:10152000EC01FC01E859FF4F1082379781E080837E
:1015300060E08D8150DC8F859889892B29F060E0EF
:101540008B85DF91CF9147CCDF91CF910895CF93D9
:10155000DF93EC018B8917DC892B11F08E8901C098
:1015600080E0DF91CF910895CF93DF93EC018989DB
:101570000ADC892B11F08E8901C080E0DF91CF91C8
:101580000895603E710508F00DC2FB018827EC57F5
:10159000FF4F8F4F0C94EB4181E090E090935B07FD
:1015A00080935A07089510925D0710925C07089582
:1015B00010925F0710925E07089581E090E090938B
:1015C0006107809360070895109263071092620785
:1015D000089583E090E090936507809364070895F1
:1015E00088E790E09093710780937007089588E7EB
:1015F00090E09093730780937207089588E790E0D6
:10160000909375078093740708951092790710924C
:101610007807089510927B0710927A07089581E069
:1016200090E090937D0780937C07089510927F0748
:1016300010927E07089510928107109280070895F6
:1016400010928307109282070895109285071092D6
:1016500084070895109287071092860708951092C4
:10166000890710928807089510928D0710928C07B1
:10167000089510928F0710928E0708951092910787
:101680001092900708951092990710929807089564
:1016900010929B0710929A07089510929D0710923E
:1016A0009C07089581E090E09093A3078093A207A0
:1016B000089581E090E09093A5078093A407089592
:1016C0008CE291E09093AD078093AC0708958CE293
:1016D00091E09093AF078093AE0708958CE291E07C
:1016E0009093B1078093B00708951092B5071092B8
:1016F000B40708951092B7071092B6070895109294
:10170000B9071092B80708951092C1071092C00748
:1017100008951092C3071092C207089581E090E0E7
:101720009093C5078093C407089585E090E0909357
:10173000C9078093C807089585E090E09093CB0790
:101740008093CA07089589E190E09093CD07809334
:10175000CC07089582E390E09093D5078093D40757
:10176000089582E390E09093D7078093D607089579
:1017700082E390E09093D9078093D807089582E39D
:1017800090E09093DD078093DC07089582E390E07A
:101790009093DF078093DE07089582E390E09093B3
:1017A000E1078093E007089580E991E09093E907CD
:1017B0008093E807089580E991E09093EB07809388
:1017C000EA07089580E991E09093ED078093EC0794
:1017D000089510927D0810927C08089510927F0859
:1017E00010927E0808951092810810928008089542
:1017F000109225081092240808951092270810923C
:101800002608089510922908109228080895109229
:101810002D0810922C08089510922F0810922E086F
:1018200008951092310810923008089585E090E0F4
:101830009093390880933808089585E090E090935C
:101840003B0880933A08089585E090E090933D0826
:1018500080933C08089588E390E09093410880933A
:101860004008089588E390E09093430880934208ED
:10187000089588E390E09093450880934408089584
:1018800085E090E090934D0880934C08089585E0A2
:1018900090E090934F0880934E08089585E090E083
:1018A0009093510880935008089510925508109213
:1018B00054080895109257081092560808951092EF
:1018C0005908109258080895109261081092600803
:1018D00008951092630810926208089510926508A6
:1018E0001092640808951092ED081092EC08089583
:1018F0008CE390E09093EF088093EE08089581E0E8
:1019000090E09093F1088093F00808951092F50804
:101910001092F40808958CE390E09093F708809378
:10192000F608089581E090E09093F9088093F80814
:101930000895109201091092000908958CE390E037
:101940009093030980930209089581E090E09093B9
:101950000509809304090895109209091092080955
:1019600008958CE390E090930B0980930A09089501
:1019700081E090E090930D0980930C0908951092F6
:1019800015091092140908958CE390E090931709BB
:1019900080931609089581E090E09093190980934F
:1019A00018090895660F771FFB01E65AF84F118258
:1019B000108208958FEF9FEF08958BE794E00E94C7
:1019C000E53681E193E00E94E5360E941A220E94EA
:1019D000392180E090E008950C94BE440C94BE44FC
:1019E0000C94BE440C94BE440C94BE440C94BE446F
:1019F0000C94BE440C94BE440C94BE440C94BE445F
:101A00000C94BE448F929F92AF92BF92CF92DF927E
:101A1000EF92FF920F931F93CF935FD7C1E0CF93C5
:101A20001F921F921F921F92812C912CA12CB12CDE
:101A3000C12CD12C760197018601B701A6010E9425
:101A4000EB164BD71F92CF93CF931F921F92970104
:101A50008601B701A6010E94EB168DB79EB70A96C4
:101A60000FB6F8949EBF0FBE8DBF80E090E0CF917F
:101A70001F910F91FF90EF90DF90CF90BF90AF90AC
:101A80009F908F9008954F925F926F927F928F9266
:101A90009F92AF92BF92CF92DF92EF92FF920F93FD
:101AA0001F93CF93DF9300D01F92CDB7DEB7FB011A
:101AB0001689078982889388A684B784C284D384D0
:101AC000E484F58446805780608471844281538128
:101AD0006481758149835A836B837C83FED61F9210
:101AE0001F921F920F931F939301820149815A8184
:101AF0006B817C810E94EB160F900F900F900F90DE
:101B00000F9080E090E00F900F900F900F90DF917A
:101B1000CF911F910F91FF90EF90DF90CF90BF90EA
:101B2000AF909F908F907F906F905F904F900895AF
:101B3000CF93DF93EB0120E030E040E85FE36A8180
:101B40007B818C819D810E94D049811112C080E8E7
:101B500094E00E94E536C1D6FC01E35BFF4F1082A2
:101B6000118212821382E25DFE4F108A118A128A5C
:101B7000138A20E030E040E85FE36E817F81888552
:101B800099850E94D049811112C080E994E00E9499
:101B9000E536A3D6FC01EA53FF4F10821182128270
:101BA0001382E153FF4F108A118A128A138A20E0B0
:101BB00030E040E85FE36A857B858C859D850E94E7
:101BC000D049811112C080EA94E00E94E53685D6A2
:101BD000FC01E15CFE4F1082118212821382E059F7
:101BE000FF4F108A118A128A138A0E941A220E94B9
:101BF000392180E090E0DF91CF9108950E941A2270
:101C00000E948C2180E090E0089580EB94E00E9497
:101C1000E5360E941A220E9481220E941A220E9406
:101C20004B210E94361640E050E068E070E0CAD6D2
:101C30000E94361640E050E069E070E0C3D60E9492
:101C4000361640E050E06AE070E0BCD60E943616DE
:101C500040E050E06DE070E0B5D680E090E008959F
:101C60000F931F93CF93DF93FB01C2A1D3A1068DE6
:101C7000178D8091F0099091F109892B41F481E051
:101C800090E00E9429449093F1098093F009043078
:101C9000110539F00530110541F4BE018DE39BE0DB
:101CA00003C0BE018AE39BE06FDA80E090E0DF9141
:101CB000CF911F910F9108956F927F928F929F9273
:101CC000AF92BF92CF92DF92EF92FF920F931F934A
:101CD000CF93DF93FB01E2A8F3A886A497A4A0A862
:101CE000B1A8C6A0D7A062A073A0068D178DBED7DD
:101CF000EC019701A301B801D1D6C501B401B6D951
:101D00009701A601B801CE01C9D680E090E0DF912D
:101D1000CF911F910F91FF90EF90DF90CF90BF90E8
:101D2000AF909F908F907F906F9008950F931F9327
:101D3000CF93DF931F92CDB7DEB78B01000F111F3A
:101D4000642FC80159830E94F44A5981652FC80144
:101D500001960E94F44A80E090E00F90DF91CF91CD
:101D60001F910F9108950F931F93CF93DF93EB0172
:101D70009CD7882331F1FE01EE0FFF1FE65AF84F82
:101D80000081118187EB94E00E94E5368EE794E0B4
:101D90000E94E5368BEB94E00E94E536CE010E946E
:101DA00016388EE794E00E94E5368DEB94E00E94B1
:101DB000E536C8010E9416380E941A220E94392175
:101DC00004C08FEB94E00E94E53680E090E0DF9164
:101DD000CF911F910F910895BF92CF92DF92EF9212
:101DE000FF920F931F93CF93DF938091F20990910D
:101DF000F309892B09F088C084E090E00E9429440F
:101E0000EC0180E090E00E94EC4A182F81E090E025
:101E10000E94EC4A482F50E060E070E0762F652F7A
:101E2000542F4427812F90E0480F591F1416150690
:101E30006CF100E010E0B801CE0137D7882319F02B
:101E4000B801CE019EDB0F5F1F4F013E110599F7D0
:101E50006AE5E62E67E0F62E00E010E0B801CE015C
:101E600024D7882331F0F70140815181B801CE0198
:101E70005DDF0F5F1F4FF2E0EF0EF11C0639110519
:101E800069F7D093F309C093F2093EC04AE5E42E06
:101E900047E0F42ECC24C394D12C00E010E0B8012C
:101EA000CE0103D7882321F1C801880F991F0E9412
:101EB000EC4AB82EC6010E94EC4A482F50E060E080
:101EC00070E0762F652F542F44278B2D90E0480F1C
:101ED000591FF701518340834F3F5F4F49F4B801C9
:101EE000CE014FDBF70140815181B801CE011EDFE9
:101EF0000F5F1F4FF2E0EF0EF11C82E0C80ED11C05
:101F0000013E110561F6BDCF8091F2099091F30970
:101F1000DF91CF911F910F91FF90EF90DF90CF90C5
:101F2000BF90089508950895089508950895089517
:101F300008950895089508950895CF92DF92EF923D
:101F4000FF920F931F93CF93DF937C016B018A0164
:101F5000E90142DFF601EE0FFF1FE65AF84F8081DC
:101F60009181F7019183808337DF000F111FF80102
:101F7000E65AF84F81E0208131812130310509F0A6
:101F800080E0F701828728DFCC0FDD1FC65AD84FCB
:101F900088819981092E000CAA0BBB0BF701828363
:101FA0009383A483B5831682178210861186DF91EE
:101FB000CF911F910F91FF90EF90DF90CF900895F8
:101FC000CF92DF92EF92FF920F931F93CF93DF9305
:101FD000EC0186E390E09E8B8D8B87E390E0988FF9
:101FE0008F8B86E290E09A8F898F8AE190E09C8FB8
:101FF0008B8F8CE190E09E8F8D8F88E190E098A38D
:102000008F8F83E090E09AA389A382E090E09CA365
:102010008BA3FE01E757FF4F8CE390E09683858307
:102020008DE390E09087878388E390E092878187B3
:102030001486138616861586108A17868EE090E021
:10204000928B818B8FE090E0948B838BE758FF4FCE
:102050008EE290E09683858380E390E0908787838B
:102060008EE390E092878187148613861686158604
:10207000108A178682E190E0928B818B83E190E059
:10208000948B838BE852FF4F11821082329611821B
:102090001082329611821082CE010E94C822CE0197
:1020A0000E94AA2F6E0185E8C81A8EEFD80A80E137
:1020B00090E0F6019183808381E190E095838483B1
:1020C0008FE190E09383828381E290E0978386831F
:1020D000C601BCD9F60182858087838581877E0110
:1020E000FBE6EF1AFEEFFF0A87E190E0F70191832C
:1020F000808389E190E09583848383E290E09383F9
:10210000828385E290E097838683C7019FD9F70198
:1021100082858087838581878E0101551E4F8BE1E3
:1021200090E0F801918380838DE190E09583848332
:1021300087E290E09383828389E290E097838683AD
:10214000C80184D9F8018285808783858187EF5013
:10215000FF4F808191813C9720813181369740816A
:102160005181F601578B468B358B248B019719F4DF
:102170008FEF9FEF03C081E090E0F601918F808F99
:10218000FE01EE55FD4F808191813C972081318188
:10219000369740815181F701578B468B358B248BC5
:1021A000019719F48FEF9FEF03C081E090E0F701F2
:1021B000918F808FFE01EC55FD4F808191813C977E
:1021C00020813181CE56DD4F48815981F801578BEE
:1021D000468B358B248B019719F48FEF9FEF03C04B
:1021E00081E090E0F801918F808FDF91CF911F9176
:1021F0000F91FF90EF90DF90CF9008952F923F9234
:102200004F925F926F927F928F929F92AF92BF9206
:10221000CF92DF92EF92FF920F931F93CF93DF93B2
:10222000CDB7DEB7C957D1090FB6F894DEBF0FBEE0
:10223000CDBF8C01FC0110821182128213821482A4
:1022400015821682178210861186128613861486CE
:102250001586168617862C01F0E14F0E511CC2011F
:102260000E94132F680189E8C80ED11CC6010E9484
:10227000132F7801EEEFEE1AFE0AC7010E94132F0A
:102280003801F5E86F1AFEEF7F0AC30131D9480122
:102290008BE6881A8EEF980AC4012AD95801E1E525
:1022A000AE1AEEEFBE0AC50123D968EC73E0C8018F
:1022B00087539E4F0E945006F801E153FE4F118252
:1022C00010823296118210823296118210823296DA
:1022D00011821082329610823196108231961082CD
:1022E00031961182108232961182108232961182BA
:1022F0001082329610823196108231961082319679
:1023000010821182128213823496108211821282FC
:1023100013823496108211821282138234961082B4
:1023200011821282138234961082118212821382D9
:102330003496108211821282138234961082118296
:102340001282138234961082118212821382349682
:1023500010821182128213823496108211821282AC
:102360001382349610821182128213823496108264
:102370001182128213823496108231961082319625
:10238000108231961082118212821382349610824A
:102390001182128213823496108211821282138269
:1023A00034961082319610823196108231961082C6
:1023B00031961082319610823196108231961082B9
:1023C00031961082319610823196108231961082A9
:1023D0003196108231961082319610823196108299
:1023E0003196108231961082319610823196108289
:1023F00031961082319610821182128213823496A5
:1024000010821182128213823496108211821282FB
:102410001382D801AD5BBD4F8CE0EAE1F3E001909F
:102420000D928A95E1F7F801E15BFD4F1082118270
:102430001282138234961082118212821382349691
:102440001082118212821382349611821082329687
:10245000118210823296118210823296108211827D
:102460001282138234961082118212821382349661
:10247000108211821282138234961082118212828B
:102480001382349610821182128213823496108243
:102490001182128213823496118210823296118236
:1024A000108232961182108232961082118212822C
:1024B0001382349610821182128213823496108213
:1024C00011821282138234961082319610823196D4
:1024D00010823196118210823296118210823296C9
:1024E00011821082329611821082329611821082ED
:1024F00032961182108232961182108232961182A7
:102500001082329611821082329611821082329697
:1025100011821082329611821082329611821082BC
:102520003296118210821801F6E52F1AFDEF3F0A4C
:10253000F1011082CE0101960E94132F89E7FE015E
:102540003196D20101900D928A95E1F7CE01019664
:102550000E94132F89E7FE013196D60101900D925A
:102560008A95E1F7CE0101960E94132F89E7FE01BB
:102570003196D70101900D928A95E1F788E5F8012F
:10258000808B89E5F60180838AE5F7018083CE019F
:1025900001960E94780A8AE1FE013196D3010190EA
:1025A0000D928A95E1F7CE0101960E94780A8AE1A0
:1025B000FE013196D40101900D928A95E1F7CE018A
:1025C00001960E94780A8AE1FE013196D5010190B8
:1025D0000D928A95E1F7C801F3DCF1011082C7582A
:1025E000DF4F0FB6F894DEBF0FBECDBFDF91CF91A6
:1025F0001F910F91FF90EF90DF90CF90BF90AF9021
:102600009F908F907F906F905F904F903F902F9012
:1026100008950F931F93CF93DF938B01EA0182E319
:1026200093E00E94E5368EE794E00E94E536F801DB
:1026300080810E942637CE010E9416380E941A22FD
:10264000DF91CF911F910F910C943921CF92DF929E
:10265000EF92FF920F931F93CF93DF93CDB7DEB727
:1026600028970FB6F894DEBF0FBECDBF8B016A016D
:1026700087539E4F7C016EE273E00E9412066EE764
:1026800074E0C7010E941206F801808189831A82D2
:1026900041E050E08E010F5F1F4FB801C7010E945B
:1026A000B5054AE0B801C6010E948345F8010190D2
:1026B0000020E9F73197AF01401B510BB801C7016A
:1026C0000E94B5050E941A22BC01C8010E94F32095
:1026D000B801C7010E94200689819A810E94BE44E8
:1026E00028960FB6F894DEBF0FBECDBFDF91CF9115
:1026F0001F910F91FF90EF90DF90CF900895FC0114
:10270000DB01AE59BF4F8C91882319F022E030E0F5
:1027100002C020E030E0DB01AC59BF4F8C91882330
:1027200011F023E030E0DB01AD59BF4F8C918823DD
:1027300011F024E030E0DB01AB59BF4F8C918823CE
:1027400011F026E030E0DA018D919C918217930719
:1027500021F091E0121613060CF090E0DA012D93AF
:102760003C93992319F0A901CF0170CF08958F925E
:102770009F92AF92BF92CF92DF92EF92FF920F9310
:102780001F93CF93DF93EC018AE293E00E94E5363A
:102790008DE894E00E94E5366E0185E8C81A8EEF58
:1027A000D80AC6010E94590A0E94D6494B015C0111
:1027B000FE01ED5BFD4F60817181828193810E94FA
:1027C000D6499B01AC01C501B4010E945F420E9441
:1027D00058378DE994E00E94E5367E01EBE6EE1A6B
:1027E000EEEFFE0AC7010E94590A0E94D6494B012A
:1027F0005C01FE01E95BFD4F608171818281938103
:102800000E94D6499B01AC01C501B4010E945F4200
:102810000E9458378DEA94E00E94E5368E010155FA
:102820001E4FC8010E94590A0E94D6494B015C0103
:10283000C55BDD4F688179818A819B810E94D64981
:102840009B01AC01C501B4010E945F420E94583750
:102850000E941A220E94392186E293E00E94E53606
:102860008DE894E00E94E536F601A08DB18D2089B7
:102870003189428953890E94284B0E9431378DE962
:1028800094E00E94E536F701A08DB18D2089318951
:10289000428953890E94284B0E9431378DEA94E087
:1028A0000E94E536F801A08DB18D208931894289D9
:1028B00053890E94284B0E9431370E941A22DF91CF
:1028C000CF911F910F91FF90EF90DF90CF90BF902D
:1028D000AF909F908F900C943921CF93DF9380918C
:1028E000F8099091F909892B51F48BEA92E00E9442
:1028F0002944EC0183DCD093F909C093F809809155
:10290000F8099091F909DF91CF910895CF93DF9362
:10291000EC012AEC30E04BEC50E069EC70E00DDBB0
:102920002EEC30E04FEC50E06DEC70E0CE010C96F8
:1029300004DB24ED30E045ED50E063ED70E0CE01C6
:102940004896FBDA28ED30E049ED50E067ED70E0A5
:10295000CE018496F2DA2EED30E04FED50E06DEDD1
:1029600070E0CE01C096DF91CF91E7CACF93DF939D
:102970008091F6099091F709892BE9F48CE390E0B6
:102980000E942944EC01FC01CC96118210823C96F5
:10299000E817F907D1F7198218821D861C86198E4F
:1029A000188E1DA21CA219AA18AACE01AFDFD093BF
:1029B000F709C093F6098091F6099091F709DF9124
:1029C000CF910895EF92FF920F931F93CF93DF93D0
:1029D000162F072F7A014115510559F4862F0E94B1
:1029E000C30631E020E0019709F030E0C32FD22F79
:1029F00026C04130510509F5262F663310F02AEC28
:102A0000260F80917B00922F9870877F892B80936F
:102A10007B002770206420937C0080917A00806482
:102A200080937A0080917A0086FDFCCFC091780077
:102A300080917900D0E0D82B02C0C0E0D0E082E0E5
:102A4000E816F10410F581EE94E00E94E5368EE779
:102A500094E00E94E5368BEB94E00E94E536812FEE
:102A6000902F0E9416388EE794E00E94E5368DEB99
:102A700094E00E94E536CE010E9416380E941A2288
:102A80000E94392180E090E002C081E090E0DF9177
:102A9000CF911F910F91FF90EF9008950F931F9387
:102AA000CF93DF938B01EA01AB01415051094433CD
:102AB000510508F0D4C02230310508F0D0C048E3F9
:102AC000429FF001439FF00D1124E60FF71FE80F1E
:102AD000F91F81E08083232B11F46C2F07C061E084
:102AE000802F0E94EF07209739F460E0802F0E942A
:102AF000EB0680E090E0B5C0CF3FD10509F4ADC052
:102B0000F801E451FD4FE4918E2F90E0FC013197E4
:102B1000E231F10508F09DC08827EC59FE4F8F4F38
:102B20000C94EB4184B5806884BDC7BDE2CF84B509
:102B3000806284BDC8BDDDCF8091800080688093B5
:102B40008000D0938900C0938800D3CF809180000B
:102B5000806280938000D0938B00C0938A00C9CF9D
:102B600080918000886080938000D0938D00C09316
:102B70008C00BFCF8091B00080688093B000C0937C
:102B8000B300B7CF8091B00080628093B000C09353
:102B9000B400AFCF80919000806880939000D09374
:102BA0009900C0939800A5CF809190008062809397
:102BB0009000D0939B00C0939A009BCF809190008F
:102BC000886080939000D0939D00C0939C0091CF2B
:102BD0008091A00080688093A0008091A0008F7BEE
:102BE0008093A000D093A900C093A80082CF8091C9
:102BF000A00080628093A000D093AB00C093AA0095
:102C000078CF8091A00088608093A000D093AD0021
:102C1000C093AC006ECF809120018068809320012A
:102C2000D0932901C093280164CF80912001806254
:102C300080932001D0932B01C0932A015ACF809119
:102C40002001886080932001D0932D01C0932C0136
:102C500050CFC038D1050CF448CF61E047CF81E0B8
:102C600090E0DF91CF911F910F9108958091F40929
:102C70009091F509892BA1F480E790E00E94294406
:102C8000FC01F9969C0123593F4FDF01D8971C9214
:102C90001192E217F307C9F79093F5098093F409AD
:102CA0008091F4099091F5090895683671050CF04A
:102CB00050C0653671050CF08CC06C32710554F54E
:102CC000693271050CF085C06831710594F46F307C
:102CD00071050CF07EC06630710544F462307105F8
:102CE0000CF077C0672B09F072C073C06B5071098C
:102CF0006BC0623271053CF46F3171050CF069C034
:102D00006951710961C0645271096230710508F03E
:102D10005EC05FC06A3371057CF4673371050CF0E7
:102D200058C06D3271050CF452C0603371050CF45B
:102D300050C06353710948C0643471053CF4613478
:102D400071050CF046C06D5371093EC0675471099E
:102D50003BC060397105F4F46D387105D4F5663700
:102D6000710564F463377105A4F5693671057CF16A
:102D70006C36710574F16F56710926C060387105A3
:102D800034F46D3771052CF5695771091DC063580E
:102D900071091AC0603D710564F46D3C7105CCF495
:102DA00061397105A4F0643971059CF0695C7109A1
:102DB0000BC06A3D710534F4673D710554F4635DE1
:102DC000710902C06D5D71096330710510F080E01A
:102DD000089581E008952F923F924F925F926F92F3
:102DE0007F928F929F92AF92BF92CF92DF92EF929B
:102DF000FF920F931F93CF93DF93CDB7DEB7E0978A
:102E00000FB6F894DEBF0FBECDBF1C012A013B01F7
:102E10000F83188729873A8728960EAD1FAD28970C
:102E2000FC01ED5BFD4F60817181828193810E9485
:102E3000D6499B01AC01C301B2010E94354A0E94F0
:102E4000CF426B8B7C8B8D8B9E8BF101E95BFD4FB1
:102E500060817181828193810E94D6499B01AC017E
:102E60006F81788589859A850E94354A0E94CF4274
:102E70006F8B788F898F9A8FF101E55BFD4F6081B1
:102E80007181828193810E94D6499B01AC01C70167
:102E9000B6010E94354A0E94CF426B8F7C8F8D8F86
:102EA0009E8F0E946E086F87788B898B9A8BF101B9
:102EB000ED52FE4F11821082329611821082A114BF
:102EC000B10489F0C501A0E0B0E03E964081518197
:102ED0006281738184179507A607B70724F480835E
:102EE0009183A283B3838114910491F0A12CB12C1E
:102EF000F101E951FE4F80819181A281B381881651
:102F00009906AA06BB0624F480829182A282B3822B
:102F10000115110591F020E030E0F101E551FE4F7F
:102F200080819181A281B381081719072A073B0785
:102F300024F400831183228333839101205F3F4F68
:102F40003E872D87F101ED51FE4F80819181A28155
:102F5000B381F10187A390A7A1A7B2A72101F9E846
:102F60004F0E511CF101E951FE4F80819181A281E8
:102F7000B381F201878B908FA18FB28F3101FEEF69
:102F80006F1A7F0AF101E551FE4F80819181A28184
:102F9000B381F301878B908FA18FB28F0E941A2289
:102FA0000E941A220E941A220E941A22409120098D
:102FB0005091210960912209709123094DA75EA7C4
:102FC0006FA778AB0E941A2280912409909125095D
:102FD000A0912609B09127098F839887A987BA877E
:102FE0000E941A228090280990902909A0902A090D
:102FF000B0902B09F101E15BFD4F1082118212822A
:1030000013823496108211821282138234961082B7
:1030100011821282138234961182108232961182AA
:10302000108232961182108232964DA55EA56FA550
:1030300078A9408351836283738334968F81988506
:10304000A985BA8580839183A283B38334968082D5
:103050009182A282B3822996EFAC29970B891C89B1
:103060002D893E898D859E850E94A02A2A96EFACE7
:103070002A970F89188D298D3A8D4F81588569853A
:103080007A85C2010E94A02A2B96EFAC2B970B8D5C
:103090001C8D2D8D3E8DB501A401C3010E94A02A77
:1030A000D10151961C92F101E657FF4F1082E7586B
:1030B000FF4F1082C1010E94772FC1010E947B2F18
:1030C0008D859E850E94F12EC2010E94F12EC301C2
:1030D0000E94F12E81E090E0F101E652FE4F9183D3
:1030E00080837101B4E2EB1ABEEFFB0AF701918312
:1030F0008083810102521E4FD8018D939C9341E041
:1031000050E06D857E85C101A1DAF70140815181D2
:10311000B201C1019BDAD8014D915C91B301C101AB
:1031200095DA11E0F101E655FD4F10838D859E85FE
:103130000E948B2AC2010E948B2AC3010E948B2A03
:1031400064E670E080E090E00E943608C101895298
:103150009E4FFC011083D101A852BE4F1C93A101C8
:1031600047525E4FFA0110832996FFAD2997F1115E
:103170000FC02A962FAD2A97211105C02B963FAD7F
:103180002B97332339F1910122593F4FF9011082D6
:103190002A96FFAD2A97F11105C0910129513F4FA1
:1031A000F90110822B96FFAD2B97F11105C091010B
:1031B000205A3E4FF901108229962FAD2997FC0124
:1031C00020832A963FAD2A973C932B96EFAD2B9701
:1031D000DA01EC938D859E850E944C2CC2010E94E1
:1031E0004C2CC3010E944C2C8D859E850E94A12BE6
:1031F000C2010E94A12BC3010E94A12B0E941A228E
:10320000DC0116968C918B8B18861F82F101E95296
:10321000FE4FF88FEF8B910128523E4F3C8F2B8F42
:10322000A10147525E4F58A34F8FC10186529E4F56
:1032300098A78FA3D101A452BE4FBAA7A9A73796CA
:10324000FCA7EBA7275631403EA32DA34351514085
:103250005AA349A38B5991099CA38BA3AF89B88D1D
:103260008C9181110BC0EB8DFC8D8081811106C08A
:10327000AF8DB8A18C91882309F460C3BB89B111CB
:103280005DC34FA158A56D857E85C10138DA49A57A
:103290005AA5B201C10133DA4BA55CA5B301C10146
:1032A0002EDA8D859E850E940B2CC2010E940B2C6C
:1032B000C3010E940B2CADA1BEA18C91882349F1C2
:1032C0008D859E850E944C2C4101B5E78B1ABDEF80
:1032D0009B0A5101E1E8AE1AEDEFBE0A6101F6E684
:1032E000CF1AFDEFDF0A710123E9E21A2DEFF20A8E
:1032F00081010F591D4F9101215B3D4FA10145589F
:103300005E4F6D857E85C1010E948329ADA1BEA15E
:103310001C92F101E651FF4FFC87EB8780818823E7
:1033200039F1C2010E944C2C4101F4E78F1AFDEFE4
:103330009F0A51012DE7A21A2DEFB20A610134E66E
:10334000C31A3DEFD30A71014FE8E41A4DEFF40AB6
:1033500081010B591D4F91012D5A3D4FA1014B5633
:103360005E4FB201C1010E948329AB85BC851C92CE
:10337000F101ED59FE4FFC87EB878081882339F1FD
:10338000C3010E944C2C4101F3E78F1AFDEF9F0A05
:10339000510129E7A21A2DEFB20A610132E6C31AE0
:1033A0003DEFD30A71014BE8E41A4DEFF40A8101B5
:1033B00007591D4F9101295A3D4FA10141555E4FBB
:1033C000B301C1010E948329AB85BC851C92810198
:1033D00002591F4FF8018081882309F43EC0E55F40
:1033E000FD4F60817181072E000C880B990B0E94A4
:1033F000D6499B01AC01F101E15BFD4F6081718118
:10340000828193810E94014318163CF5D8011C92D9
:103410006AE474E0810107531E4FC8010E9412063E
:1034200063E275E0C8010E94120666EC73E0C80111
:103430000E9412062996BFAD2997BB2309F479C3D0
:10344000F101E558FE4F108A118A128A138AEE5252
:10345000F1401082118212821382810109511F4FA3
:10346000D8018C91882309F43FC0F101E558FD4F44
:1034700060817181072E000C880B990B0E94D64940
:103480009B01AC01F101ED5AFD4F60817181828198
:1034900093810E94014318163CF5D8011C926AE4FE
:1034A00074E0810107531E4FC8010E9412066BE4AD
:1034B00075E0C8010E94120666EC73E0C8010E9424
:1034C00012062A96BFAD2A97BB2309F437C3F10130
:1034D000EB56FE4F108A118A128A138AE9A1FAA1CB
:1034E00010821182128213828101005A1E4FD8016C
:1034F0008C91882309F43FC0F101E358FD4F6081AE
:103500007181072E000C880B990B0E94D6499B01F4
:10351000AC01F101E95AFD4F608171818281938193
:103520000E94014318163CF5D8011C926AE474E02D
:10353000810107531E4FC8010E94120663E775E020
:10354000C8010E94120666EC73E0C8010E941206D0
:103550002B96BFAD2B97BB2309F4F5C2F101E155C2
:10356000FE4F108A118A128A138AEBA1FCA11082E5
:1035700011821282138260E08D859E850E94162B37
:10358000882369F0F101E35BFF4F10821182128200
:103590001382E25DFE4F108A118A128A138A60E05C
:1035A000C2010E94162B882371F0A9A1BAA11D9215
:1035B0001D921D921C921397F101EB56FE4F108A3B
:1035C000118A128A138A60E0C3010E94162B882395
:1035D00069F0EBA1FCA11082118212821382F10129
:1035E000E155FE4F108A118A128A138AF101E259BD
:1035F000FF4F8081AF89B88D8C93E758FF4F808152
:10360000EB8DFC8D8083F101E05AFE4F8081AF8D00
:10361000B8A18C93E351F140408151816281738163
:10362000E9A1FAA180809180A280B380ABA1BCA166
:10363000CD90DD90ED90FC904DA75EA76FA778AB85
:10364000F9D64DA55EA56FA578A9409320095093A2
:1036500021096093220970932309ECD680922409F2
:1036600090922509A0922609B0922709E3D6C0922C
:103670002809D0922909E0922A09F0922B09C10168
:103680000E94772FEF89F88D8081882309F44AC042
:103690000E946E082F85388949895A8962177307F5
:1036A0008407950760F40E946E082F853889498940
:1036B0005A896217730784079507A0F51EC00E94F8
:1036C0006E086B017C012F85388949895A89C21A95
:1036D000D30AE40AF50AF101E95CFD4F208131814A
:1036E00042815381A8EEB3E00E941E4B6C157D050C
:1036F0008E059F0508F42CC2D6CF0E946E086B0180
:103700007C01F101E95CFD4F2081318142815381CF
:10371000A8EEB3E00E941E4B6C157D058E059F053B
:1037200008F416C2AB8DBC8D8C91882309F44AC075
:103730000E946E082F85388949895A896217730754
:103740008407950760F40E946E082F85388949899F
:103750005A896217730784079507A0F51EC00E9457
:103760006E086B017C012F85388949895A89C21AF4
:10377000D30AE40AF50AF101E95CFD4F20813181A9
:1037800042815381A8EEB3E00E941E4B6C157D056B
:103790008E059F0508F4E8C1D6CF0E946E086B0124
:1037A0007C01F101E95CFD4F20813181428153812F
:1037B000A8EEB3E00E941E4B6C157D058E059F059B
:1037C00008F4D2C1AF8DB8A18C91882309F44AC006
:1037D0000E946E082F85388949895A8962177307B4
:1037E0008407950760F40E946E082F8538894989FF
:1037F0005A896217730784079507A0F51EC00E94B7
:103800006E086B017C012F85388949895A89C21A53
:10381000D30AE40AF50AF101E95CFD4F2081318108
:1038200042815381A8EEB3E00E941E4B6C157D05CA
:103830008E059F0508F4A4C1D6CF0E946E086B01C7
:103840007C01F101E95CFD4F20813181428153818E
:10385000A8EEB3E00E941E4B6C157D058E059F05FA
:1038600008F48EC184E09AE00E942203181619061B
:103870005CF584E09AE00E9400038F7D8534910519
:1038800019F565EE74E0C10187539E4F0E94120640
:1038900082E493E00E94E536CDD5EBD4F101E25904
:1038A000FF4F1082E758FF4F1082E758FF4F1082FA
:1038B000AF89B88D1C92EB8DFC8D1082AF8DB8A1B5
:1038C0001C92B1E0BB8B04C0EF81F8853197A9F45D
:1038D0006AEF74E0C10187539E4F0E941206AF89C0
:1038E000B88D1C92EB8DFC8D1082AF8DB8A11C920F
:1038F000E1E0F0E0F887EF8302C018861F82C10183
:103900000E949B36F101EB52FE4F8081918101961E
:10391000918380838D3291400CF4A0CCD101A353CC
:10392000BE4F8D919C911197892B09F097CC1496DD
:103930008D919C91892B09F42FC190CC8101035367
:103940001E4FF80180819181892B21F0C1010E94D5
:103950009B36F7CF8AE095E00E94E5362996FFADC9
:103960002997FF23F1F02F813885232BD1F43B8950
:1039700031113CC08EE393E00E94E5365BD579D4EB
:103980002A964FAD2A97442361F18AE393E00E947F
:10399000E53650D56ED42B965FAD2B9751111AC0DA
:1039A00025C02A968FAD2A97882341F0AF81B8852C
:1039B000AB2B21F4BB89B11119C0E7CF2B96EFAD2A
:1039C0002B97EE2399F02F813885232B79F43B89AF
:1039D00031110CC086E393E00E94E5362BD549D423
:1039E00005C02B96AFAD2B97A111F4CF81010652E4
:1039F0001E4F85E090E0D8018D939C936101B4E265
:103A0000CB1ABEEFDB0AF601918380837101F2E2EB
:103A1000EF1AFEEFFF0AD7018D939C9345E050E02B
:103A20006D857E85C1010E942613F601408151817A
:103A3000B201C1010E942613D7014D915C91B301DF
:103A4000C1010E942613C1010E947F2FF101E35B97
:103A5000FF4F4081518162817381E758FF4F808021
:103A60009180A280B380E758FF4F80819181A2812D
:103A7000B3818F87988BA98BBA8B4DA75EA76FA751
:103A800078ABD8D44DA55EA56FA578A94093200941
:103A9000509321096093220970932309CBD480921B
:103AA000240990922509A0922609B0922709C2D430
:103AB0002F85388949895A89209328093093290903
:103AC00040932A0950932B09C1010E94772FC1010D
:103AD0000E947B2FAFD420D4C1010E94B713D8011C
:103AE0001D921C92F60111821082D7011D921C9228
:103AF00040E050E06D857E85C1010E942613F601ED
:103B000040815181B201C1010E942613D7014D911C
:103B10005C91B301C1010E942613C1010E947F2F55
:103B2000BB89BB2309F426C185D421E0FC0126838F
:103B300021C1E1E0F0E0F887EF838FCCE1E0F0E035
:103B4000F887EF83D1CCE1E0F0E0F887EF8313CD85
:103B50006BE975E0C10187539E4F0E94120621E078
:103B600030E038872F83DECD60EB75E0C1018753ED
:103B70009E4F0E94120641E050E058874F8322CEAC
:103B800065EC75E0C10187539E4F0E94120681E0EB
:103B900090E098878F8366CE11821082F101ED52FA
:103BA000FE4FE080F180E114F10449F466E473E033
:103BB000810107531E4FC8010E941206B8C091E050
:103BC000E916F10409F0C2C035D48C01DC018D91F5
:103BD0009C9111971816190614F0ED92FC92F801B9
:103BE000828193811816190624F081E090E0938376
:103BF0008283D80114968D919C91159718161906F9
:103C000034F081E090E015969C938E93149768ECC5
:103C100073E0CE0101960E94500666E075E0CE0189
:103C200001960E9412066DE874E0CE0101960E9492
:103C300012066091200970912109809122099091CA
:103C400023090E94D6496B017C01F80160817181D2
:103C5000072E000C880B990B0E94D6499B01AC01E2
:103C6000C701B6010E945F42AB01BC01CE010196C3
:103C70000E94E2056DE974E0CE0101960E941206F1
:103C80006091240970912509809126099091270956
:103C90000E94D6496B017C01D80112966D917C91EE
:103CA0001397072E000C880B990B0E94D6499B0195
:103CB000AC01C701B6010E945F42AB01BC01CE015D
:103CC00001960E94E2056DEA74E0CE0101960E9421
:103CD0001206609128097091290980912A09909112
:103CE0002B090E94D6496B017C01F8016481758122
:103CF000072E000C880B990B0E94D6499B01AC0142
:103D0000C701B6010E945F42AB01BC01CE01019622
:103D10000E94E205BE016F5F7F4F810107531E4F76
:103D2000C8010E94200689819A810E94BE4482D3E4
:103D3000BC01CE01019657D2BE016F5F7F4FC80113
:103D40000E94200689819A810E94BE44F101ED52B1
:103D5000FE4F808191810196823091051CF4918300
:103D6000808302C011821082F101EF52FE4F118256
:103D7000108274CA88E195E00E94E5368F819885AB
:103D80000E94163886EC93E00E94E53653D32F81CB
:103D900038853093590720935807C901E0960FB62C
:103DA000F894DEBF0FBECDBFDF91CF911F910F9171
:103DB000FF90EF90DF90CF90BF90AF909F908F904B
:103DC0007F906F905F904F903F902F9008951F933A
:103DD000CF93DF931F92CDB7DEB7FB0162A9168D9B
:103DE00069830E9436166981812F0E94EF0780E067
:103DF00090E00F90DF91CF911F9108950C94BE44F5
:103E00000C94BE440C94BE440C94BE440C94BE442A
:103E10000C94BE440C94BE440C94BE440C94BE441A
:103E20000C94BE440C94BE440C94BE440F931F9358
:103E3000CF93DF93FB0102A913A9C68DD78D0E94F2
:103E40003616A801BE010E94E21480E090E0DF91E6
:103E5000CF911F910F910895EF92FF920F931F93AF
:103E6000CF93DF93FB01E2A8F3A802A113A1C68DB3
:103E7000D78D0E9436169701A801BE010E944E15EB
:103E800080E090E0DF91CF911F910F91FF90EF9034
:103E90000895662319F087ED93E002C080ED93E06A
:103EA0000C94E536CF93DF93FB01C68DD78D0E942E
:103EB000EC0EBE010E94B30E80E090E0DF91CF9146
:103EC0000895CF92DF92EF92FF920F931F93CF93BB
:103ED000DF93FB01C2A0D3A0E4A0F5A0068D178D4F
:103EE0000E94EC0EEC018A819B818F30F7E29F07E4
:103EF00024F401969B838A8302C01B821A82B80134
:103F0000CE010E945516882389F0F801EE0FFF1F9D
:103F1000E65AF84FD182C082A601B801CE010E94B4
:103F2000960EB801CE010E94B30E04C08FEB94E050
:103F30000E94E5360E94B6140E94861480E090E04C
:103F4000DF91CF911F910F91FF90EF90DF90CF9075
:103F500008958F929F92AF92BF92CF92DF92EF928D
:103F6000FF920F931F930E946D1462E070E00E9415
:103F70007331892BD1F40E946D1421E02F931F928D
:103F80001F921F921F92812C912CA12CB12CC12C1D
:103F9000D12C760197018601B701A6010E94EB168C
:103FA0000F900F900F900F900F9080E090E01F9176
:103FB0000F91FF90EF90DF90CF90BF90AF909F90C8
:103FC0008F9008958F929F92AF92BF92CF92DF927F
:103FD000EF92FF920F931F930E946D1461E070E0C7
:103FE0000E947331892BD1F40E946D141F9221E03D
:103FF0002F931F921F921F92812C912CA12CB12CD8
:10400000C12CD12C760197018601B701A6010E942F
:10401000EB160F900F900F900F900F9080E090E0B4
:104020001F910F91FF90EF90DF90CF90BF90AF90D6
:104030009F908F9008958F929F92AF92BF92CF9250
:10404000DF92EF92FF920F931F930E946D1460E036
:1040500070E00E947331892BD1F40E946D141F927D
:104060001F9221E02F931F921F92812C912CA12C43
:10407000B12CC12CD12C760197018601B701A60184
:104080000E94EB160F900F900F900F900F9080E012
:1040900090E01F910F91FF90EF90DF90CF90BF9035
:1040A000AF909F908F9008958F929F92AF92BF9202
:1040B000CF92DF92EF92FF920F931F930E946D14A5
:1040C00021E02F931F921F921F921F92812C912CFF
:1040D000A12CB12CC12CD12C760197018601B701FE
:1040E000A6010E94EB160F900F900F900F900F906B
:1040F00080E090E01F910F91FF90EF90DF90CF90C4
:10410000BF90AF909F908F9008958F929F92AF92A3
:10411000BF92CF92DF92EF92FF920F931F930E9474
:104120006D141F9221E02F931F921F921F92812CDA
:10413000912CA12CB12CC12CD12C76019701860198
:10414000B701A6010E94EB160F900F900F900F90F1
:104150000F9080E090E01F910F91FF90EF90DF9023
:10416000CF90BF90AF909F908F9008958F929F9225
:10417000AF92BF92CF92DF92EF92FF920F931F9375
:104180000E946D141F921F9221E02F931F921F9285
:10419000812C912CA12CB12CC12CD12C7601970112
:1041A0008601B701A6010E94EB160F900F900F90A9
:1041B0000F900F9080E090E01F910F91FF90EF9093
:1041C000DF90CF90BF90AF909F908F90089508950B
:1041D00008950895089508950895089508950895F7
:1041E000089508950895EF92FF920F931F93CF9330
:1041F000DF93CDB7DEB72E970FB6F894DEBF0FBEB4
:10420000CDBF8C0168EC73E00E9450066AED75E04A
:10421000C8010E94120660911C0970911D098091CD
:104220001E0990911F092AE0AE014F5F5F4F7A018E
:104230000E948D45F70101900020E9F73197AF0109
:104240004E195F09B701C8010E94B50566EC73E01D
:10425000C8010E941206C8012E960FB6F894DEBF60
:104260000FBECDBFDF91CF911F910F91FF90EF90C7
:1042700008958AED95E00E94E53660911C097091E1
:104280001D0980911E0990911F090E94313786EC0B
:1042900093E00C94E5360F931F93CF93DF93EC01DB
:1042A0008DED95E00E94E53681EE95E00E94E536C1
:1042B0000EEF19E0F8016081CE01EBDD85EE95E0AF
:1042C0000E94E536F8016181CE01E3DD89EE95E0DB
:1042D0000E94E536F8016281CE01DBDD8DEE95E0CE
:1042E0000E94E536F8016381CE01D3DD81EF95E0D0
:1042F0000E94E536F8016481CE01CBDD85EF95E0C3
:104300000E94E536F8016581CE01C3DDCE01DF9163
:10431000CF911F910F91ADCFCF92DF92EF92FF928D
:10432000CF93DF93EC01888199811816190624F048
:1043300081E090E0998388838A819B811816190611
:1043400024F081E090E09B838A838C819D81181604
:10435000190624F081E090E09D838C8386E095E04F
:104360000E94E5368DE894E00E94E53660912009D0
:104370007091210980912209909123090E94D649C8
:104380006B017C0188819981BC01990F880B990B85
:104390000E94D6499B01AC01C701B6010E945F4251
:1043A0000E9458378DE994E00E94E5366091240917
:1043B0007091250980912609909127090E94D6497C
:1043C0006B017C018A819B81BC01990F880B990B41
:1043D0000E94D6499B01AC01C701B6010E945F4211
:1043E0000E9458378DEA94E00E94E53660912809D2
:1043F0007091290980912A0990912B090E94D64930
:104400006B017C018C819D81BC01990F880B990BFC
:104410000E94D6499B01AC01C701B6010E945F42D0
:104420000E945837CE01DF91CF91FF90EF90DF903F
:10443000CF901FCF8091FC099091FD09892B91F5B8
:1044400087E090E00E942944FC0116821092200926
:104450001092210910922209109223091092240926
:104460001092250910922609109227091092280906
:104470001092290910922A0910922B091092FB0917
:104480001092FA0910921C0910921D0910921E092F
:1044900010921F0910925907109258079093FD0926
:1044A0008093FC098091FC099091FD0908950F9378
:1044B0001F93CF93DF930E94EC0E8C01C0E0D0E0FD
:1044C000BE01C8010E945516882321F0BE01C80113
:1044D0000E94B30E2196C13ED10591F789EF95E078
:1044E0000E94E536A7DFC5DE80E090E0DF91CF9146
:1044F0001F910F9108959EDFFC01168280E090E0ED
:104500000895CF93DF9383E00E94C306EC0192DF0E
:1045100091E0CD2B09F490E09093FE0982E00E9497
:10452000C306EC0187DF91E0CD2B09F490E0909376
:10453000FF098EE00E94C306EC017CDF91E0CD2BE9
:1045400009F490E09093000A8FE00E94C306EC010A
:1045500071DF91E0CD2B09F490E09093010A82E1A4
:104560000E94C306EC0166DF91E0CD2B09F490E0D8
:104570009093020A83E10E94C306EC015BDF91E0A5
:10458000CD2B09F490E09093030ADF91CF91089529
:104590002F923F924F925F926F927F928F929F9253
:1045A000AF92BF92CF92DF92EF92FF920F931F9341
:1045B000CF93DF93CDB7DEB72F970FB6F894DEBF5A
:1045C0000FBECDBF9F878E870E94EC0EEE85FF85C4
:1045D000E052FE4F81E02091C0073091C107232BAC
:1045E00009F480E080830E94EC0EEE85FF85EF5198
:1045F000FE4F81E02091C2073091C307232B09F4BD
:1046000080E080830E94EC0EEE85FF85EE51FE4F28
:1046100081E02091C4073091C507232B09F480E085
:1046200080830E94EC0EEE85FF85ED51FE4F809158
:10463000E8079091E907092E000CAA0BBB0B8083B9
:104640009183A283B3830E94EC0EEE85FF85E9512E
:10465000FE4F8091EA079091EB07092E000CAA0B00
:10466000BB0B80839183A283B3830E94EC0EEE8503
:10467000FF85E551FE4F8091EC079091ED07092EE3
:10468000000CAA0BBB0B80839183A283B3830E948F
:10469000EC0EEE85FF85E151FE4F8091D40790919D
:1046A000D507092E000CAA0BBB0B80839183A28334
:1046B000B3830E94EC0EEE85FF85ED50FE4F809196
:1046C000D6079091D707092E000CAA0BBB0B80834D
:1046D0009183A283B3830E94EC0EEE85FF85E9509F
:1046E000FE4F8091D8079091D907092E000CAA0B94
:1046F000BB0B80839183A283B3830E94EC0EEE8573
:10470000FF85E550FE4F8091DC079091DD07092E73
:10471000000CAA0BBB0B80839183A283B3830E94FE
:10472000EC0EEE85FF85E150FE4F8091DE07909103
:10473000DF07092E000CAA0BBB0B80839183A28399
:10474000B3830E94EC0EEE85FF85ED5FFD4F8091F7
:10475000E0079091E107092E000CAA0BBB0B8083A8
:104760009183A283B3830E94EC0EEE85FF85E95FFF
:10477000FD4F8091AC079091AD07092E000CAA0B5C
:10478000BB0B80839183A283B3830E94EC0EEE85E2
:10479000FF85E55FFD4F8091AE079091AF07092E31
:1047A000000CAA0BBB0B80839183A283B3830E946E
:1047B000EC0EEE85FF85E15FFD4F8091B007909193
:1047C000B107092E000CAA0BBB0B80839183A28337
:1047D000B3830E94EC0EEE85FF85ED5EFD4F81E018
:1047E00020919807309199072130310509F080E038
:1047F00080830E94EC0EEE85FF85EC5EFD4F81E02C
:1048000020919A0730919B072130310509F080E013
:1048100080830E94EC0EEE85FF85EB5EFD4F81E00C
:1048200020919C0730919D072130310509F080E0EF
:1048300080830E94EC0EEE85FF85EF5CFD4F81E0EA
:104840002091840730918507232B09F480E0808331
:104850000E94EC0EEE85FF85EE5CFD4F81E020911D
:10486000860730918707232B09F480E080830E941C
:10487000EC0EEE85FF85ED5CFD4F81E02091880711
:1048800030918907232B09F480E080830E94EC0E8D
:10489000EE85FF85EC5CFD4F81E020918C07309127
:1048A0008D072130310509F080E080830E94EC0EF5
:1048B000EE85FF85EB5CFD4F81E020918E07309106
:1048C0008F072130310509F080E080830E94EC0ED3
:1048D000EE85FF85EA5CFD4F81E0209190073091E5
:1048E00091072130310509F080E080830E94EC0EB1
:1048F000EE85FF85E95CFD4F80917007909171070F
:10490000092E000CAA0BBB0B80839183A283B38377
:104910000E94EC0EEE85FF85E55CFD4F80917007EF
:1049200090917107092E000CAA0BBB0B8083918319
:10493000A283B3830E94EC0EEE85FF85E15CFD4F00
:104940008091700790917107092E000CAA0BBB0B88
:1049500080839183A283B3830E94EC0EEE85FF8552
:10496000EB5DFD4F81E02091780730917907232B93
:1049700009F480E080830E94EC0EEE85FF85EA5DFD
:10498000FD4F81E020917A0730917B07232B09F4BA
:1049900080E080830E94EC0EEE85FF85E95DFD4F8F
:1049A00081E020917C0730917D07232B09F480E082
:1049B00080830E94EC0EEE85FF85EA5EFD4F8091BC
:1049C000740890917508092E000CAA0BBB0B80830C
:1049D0009183A283B3830E94EC0EEE85FF85E65E91
:1049E000FD4F8091760890917708092E000CAA0B54
:1049F000BB0B80839183A283B3830E94EC0EEE8570
:104A0000FF85E25EFD4F8091780890917908092E2C
:104A1000000CAA0BBB0B80839183A283B3830E94FB
:104A2000EC0EEE85FF85E85DFD4F81E02091A40747
:104A30003091A5072130310509F080E08083EE85B3
:104A4000FF85E75DFD4F1082EE85FF85E65DFD4F3A
:104A500010820E94EC0EEE85FF85E55DFD4F81E042
:104A60002091A2073091A3072130310509F080E0A1
:104A70008083EE85FF85E45DFD4F1082EE85FF8526
:104A8000E35DFD4F10820E94EC0EEE85FF85E25D36
:104A9000FD4F81E02091B4073091B50721303105F9
:104AA00009F080E080830E94EC0EEE85FF85E15DD9
:104AB000FD4F81E02091B6073091B70721303105D5
:104AC00009F080E080830E94EC0EEE85FF85E05DBA
:104AD000FD4F81E02091B8073091B90721303105B1
:104AE00009F080E080830E94EC0EEE85FF85EE5D8C
:104AF000FD4F81E020917C0830917D082130310507
:104B000009F080E080830E94EC0EEE85FF85ED5D6C
:104B1000FD4F81E020917E0830917F0821303105E2
:104B200009F080E080830E94EC0EEE85FF85EC5D4D
:104B3000FD4F81E0209180083091810821303105BE
:104B400009F080E080830E94EC0E0E851F850D5BCE
:104B50001D4F8091C8079091C907092E000CAA0B20
:104B6000BB0BF80180839183A283B3830E94EC0E78
:104B7000EE84FF84F9EBEF1AFDEFFF0A8091CA077C
:104B80009091CB07092E000CAA0BBB0BF701808379
:104B90009183A283B3830E94EC0E8091CC07909105
:104BA000CD07092E000CAA0BBB0B2E853F85255B7C
:104BB0003D4FF90180839183A283B383F801408143
:104BC000518162817381141615061606170644F08A
:104BD00041E050E060E070E0408351836283738382
:104BE000F701408151816281738114161506160602
:104BF000170644F041E050E060E070E040835183EC
:104C000062837383181619061A061B064CF081E09E
:104C100090E0A0E0B0E0F90180839183A283B383A8
:104C2000D901CD90DC90F701E080F180D8010D91A1
:104C30001C9100DCFC0111830083F382E282D582A7
:104C4000C482EE85FF85EE5DFD4FB081B983EE85B0
:104C5000FF85EA5EFD4F80819181A281B3814E85FF
:104C60005F85425D5D4FFA01F081FB834E855F8574
:104C70004C5C5D4FFA01F081FA834E855F85485D9B
:104C80005D4FFA01F081FF834E855F85455D5D4F85
:104C9000FA01F081F8874E855F854F5C5D4FFA0120
:104CA000F081F987EE85FF85ED5EFD4F2080EE8572
:104CB000FF85E052FE4F3080EE85FF85E95CFD4FB9
:104CC0004081518162817381EE85FF85E95FFD4FEF
:104CD0000081118122813381EE85FF85E550FE4FF1
:104CE000C080D180E280F380EE85FF85E151FE4FE8
:104CF00080809180A280B380EE85FF85ED51FE4FCC
:104D00004080518062807380EE85FF8547A250A667
:104D100061A672A683A694A6A5A6B6A6C7A6D0AA83
:104D2000E1AAF2AA03AB14AB25AB36AB47AB50AF4D
:104D300061AF72AF33AE24AE298525A33A8136A385
:104D400040E450E060E070E0FF964083518362836E
:104D500073832885EE85FF8525AF3F8136AFAF0190
:104D60004D5B5F4F2B81FA012083EE85FF85EC5B65
:104D7000FF4F80839183A283B383EE85FF85E85B39
:104D8000FF4F39813083AE85BF8555968D919C91BB
:104D900056978633910589F487EB94E0FD01E75837
:104DA000FF4F9183808332961182108285EB94E0CD
:104DB000369691838083329630C08C33910589F486
:104DC0008FEA94E0EE85FF85E758FF4F918380835B
:104DD000EE85FF85E558FF4F118210828DEA94E041
:104DE00012C08E97E1F487EA94E0EE85FF85E758DC
:104DF000FF4F91838083EE85FF85E558FF4F118239
:104E0000108281EA94E0EE85FF85EF57FF4F918392
:104E10008083EE85FF85ED57FF4F11821082EE856E
:104E2000FF85838D948D4A97D1F483EB94E0E3580A
:104E3000FF4F91838083EE85FF85E158FF4F1182FC
:104E4000108281EB94E0EE85FF85EB57FF4F918355
:104E50008083EE85FF85E957FF4F11821082EE8532
:104E6000FF85ED5DFD4F20812983EE85FF85E65EA0
:104E7000FD4F4080518062807380EE85FF85E15D4B
:104E8000FD4F30813B83EE85FF85EB5CFD4F9081CC
:104E9000EE85FF85E75DFD4F40814F83EE85FF8501
:104EA000E45DFD4F50815887EE85FF85EE5CFD4F38
:104EB0008081EE85FF85EC5EFD4F2080EE85FF85CD
:104EC000EF51FE4F3080EE85FF85E55CFD4F208180
:104ED0003181428153812A873B874C875D87EE85EC
:104EE000FF85E55FFD4F4081518162817381EE85D1
:104EF000FF85E150FE4FC080D180E280F380EE85D7
:104F0000FF85ED50FE4F80809180A280B380EE85BA
:104F1000FF85E757FF4F2E853F8529513E4FD90129
:104F20000D911D912D913C91078B108F218F328F08
:104F3000838E948EA58EB68EC78ED0A2E1A2F2A2E9
:104F400043A354A365A376A32A853B854C855D8541
:104F500027A330A741A752A733A624A6858B968BFB
:104F600080E490E0A0E0B0E087A790ABA1ABB2AB4B
:104F7000388535A74F8146A75B8153AB44AA55AA14
:104F800066AA77AA898180AF85819681863391054B
:104F900089F487EB94E0AE85BF85AE50BF4F8D930B
:104FA0009C93AE85BF85AC50BF4F1D921C9285EB84
:104FB00094E026C08C33910589F48FEA94E0AE85A5
:104FC000BF85AE50BF4F8D939C93AE85BF85AC50CF
:104FD000BF4F1D921C928DEA94E012C08E97E1F4AF
:104FE00087EA94E0AE85BF85AE50BF4F8D939C930A
:104FF000AE85BF85AC50BF4F1D921C9281EA94E0F4
:10500000AE85BF85A650BF4F8D939C93AE85BF855F
:10501000A450BF4F1D921C92838594854A97D9F462
:1050200083EB94E0EE85FF85EA50FF4F9183808308
:10503000EE85FF85E850FF4F1182108281EB94E0EE
:10504000EE85FF85E250FF4F91838083EE85FF85DB
:10505000F39511821082EE85FF85EC5DFD4F908106
:1050600099832E853F85225E3D4FD9018D919D917B
:105070000D90BC91A02D8B839C83AD83BE83EE8568
:10508000FF85E05DFD4FB081BA83EE85FF85EA5C68
:10509000FD4F2080EE85FF85E65DFD4F20812F834B
:1050A000EE85FF85E35DFD4F30813887EE85FF8516
:1050B000ED5CFD4F3080EE85FF85EB5EFD4F30816E
:1050C000EE85FF85EE51FE4F2081EE85FF85E15C88
:1050D000FD4F80819181A281B381EE85FF85E15FE3
:1050E000FD4F4081518162817381EE85FF85ED5FC7
:1050F000FD4FC080D180E280F380EE85FF85E950CE
:10510000FE4F80809180A280B3800E851F850E5F48
:105110001E4FEE85FF85E551FE4F40805180628035
:105120007380F801478A508E618E728E838E948EC2
:10513000A58EB68EC78ED0A2E1A2F2A243A354A33D
:1051400065A376A387A390A7A1A7B2A723A734A797
:10515000358A268A80E490E0A0E0B0E087A790AB93
:10516000A1ABB2AB288525A73F8136A74A8143ABC7
:105170008B819C81AD81BE8184AB95ABA6ABB7AB77
:10518000298120AF858196818633910589F487EB4B
:1051900094E0EE85FF85E559FE4F91838083EE858F
:1051A000FF85E359FE4F1182108285EB94E026C003
:1051B0008C33910589F48FEA94E0EE85FF85E559FB
:1051C000FE4F91838083EE85FF85E359FE4F118268
:1051D00010828DEA94E012C08E97E1F487EA94E0A1
:1051E000EE85FF85E559FE4F91838083EE85FF852F
:1051F000E359FE4F1182108281EA94E0EE85FF852B
:10520000ED58FE4F91838083EE85FF85EB58FE4F6E
:1052100011821082D8011B968D919C911C974A9700
:10522000E1F483EB94E0EE85FF85E159FE4F918335
:105230008083EE85FF85EF58FE4F1182108281EB4F
:1052400094E0EE85FF85E958FE4F91838083EE85DB
:10525000FF85E758FE4F11821082EE85FF85EB5DDA
:10526000FD4F20818E859F854096222311F053D1DA
:1052700001C03DD1EE85FF85EA5DFD4F20818E8521
:105280009F8587579F4F222311F045D101C02FD111
:10529000EE85FF85E95DFD4F80818823D1F0C8014F
:1052A0002F960FB6F894DEBF0FBECDBFDF91CF9122
:1052B0001F910F91FF90EF90DF90CF90BF90AF9034
:1052C0009F908F907F906F905F904F903F902F9026
:1052D00022C1C8012F960FB6F894DEBF0FBECDBF16
:1052E000DF91CF911F910F91FF90EF90DF90CF90C2
:1052F000BF90AF909F908F907F906F905F904F90F6
:105300003F902F90F4C02F923F924F925F926F92F6
:105310007F928F929F92AF92BF92CF92DF92EF9245
:10532000FF920F931F93CF93DF9300D000D0CDB7A0
:10533000DEB73B011A0129011C830B83FA82E98243
:10534000DE82CD82F4018081882309F474C0F901E2
:10535000C080D180E280F38020E030E0A901C70165
:10536000B6010E940143181674F4F50120813181C1
:1053700042815381C701B6010E94F341F20160836B
:10538000718382839383F301E15AFF4F8081F1019E
:10539000008D118DC088D188E288F388E981FA8177
:1053A00080809180A280B380D801A70196018823D4
:1053B00041F00E94284B681579058A059B0544F049
:1053C00023C00E94284B86169706A806B906E4F467
:1053D000F20180809180A280B38020E030E04AEF2B
:1053E00056E4C501B4010E94D04987FF0DC020E0FA
:1053F00030E040E85FE3C501B4010E94F441F201EE
:105400006083718382839383D801A70196010E94F0
:10541000284BE981FA816083718382839383F3014E
:10542000FD9680819181A281B381EB81FC81808393
:105430009183A283B383ED81FE8180819181892B49
:1054400049F0C1010E94590AF301FD9660837183FE
:105450008283938326960FB6F894DEBF0FBECDBF2E
:10546000DF91CF911F910F91FF90EF90DF90CF9040
:10547000BF90AF909F908F907F906F905F904F9074
:105480003F902F900895CF93DF93EC018CA5882354
:1054900011F061E001C060E08F810E94EB068DA5F4
:1054A000882329F08EA5882311F061E001C060E017
:1054B0008D85DF91CF910C94EB06CF93DF93EC01B8
:1054C0008CA5882311F060E001C061E08F810E940B
:1054D000EB068DA5882329F08EA5882311F060E0C6
:1054E00001C061E08D85DF91CF910C94EB06CF93E5
:1054F000DF93EC0161E089850E94EB068DA588238E
:1055000021F061E08F850E94EB06CA59DF4F1882B7
:10551000DF91CF910895CF93DF93EC0160E089850F
:105520000E94EB068DA5882321F060E08F850E9404
:10553000EB06CA59DF4F81E08883DF91CF91089550
:10554000CF92DF92EF92FF920F931F93CF93DF934F
:10555000FC0141AF52AF63AF74AFDC01DD964D93F8
:105560005D936D937C93139714960D931D932D93D8
:105570003C931397EC01CB5BDF4FE88283A9882330
:1055800051F083A581114BC037FF05C01D921D92BC
:105590001D921C92139744A955A966A977A91416C0
:1055A00015061606170634F580AD882319F10D91FE
:1055B0001D912D913C9113976801790137FF07C028
:1055C000CC24DD247601C01AD10AE20AF30A4C1574
:1055D0005D056E057F0574F437FF07C07095609513
:1055E000509541955F4F6F4F7F4F4D935D936D93F6
:1055F0007C931397DF01A25BBF4F1D921D921D92FA
:105600001C921397E25AFF4F81E08083DF91CF9184
:105610001F910F91FF90EF90DF90CF90089510169B
:105620001106120613060CF4B1CFB5CF0F931F93DA
:10563000CF93DF938C01D62FFC01858981110BC09C
:10564000C8010E94B40AC82FC8010E94A70AD1113C
:105650000AC08C2F08C0C8010E94A70AC82FC80121
:105660000E94B40AF4CFDF91CF911F910F9108955A
:10567000CF93DF93EC01FC01E859FF4F81E0808379
:1056800039978081B297882341F080819181A281EE
:10569000B3810196A11DB11D07C080819181A281B6
:1056A000B3810197A109B10980839183A283B38358
:1056B000FE01E559FF4F20813181DE01A759BF4F1F
:1056C000C9019595879520FD03C0ED91FC910DC012
:1056D000FE01E80FF91F0190F081E02D2D913C9122
:1056E000E20FF31F0190F081E02D8C0F9D1F1995A3
:1056F0008F859889892B11F1FE01E159FF4F208197
:105700003181DE01A359BF4FC9019595879520FDD1
:1057100003C0ED91FC910DC0FE01E80FF91F01904F
:10572000F081E02D2D913C91E20FF31F0190F0816B
:10573000E02D8C0F9D1FDF91CF911994DF91CF91B8
:1057400008958F929F92AF92BF92CF92DF92EF9285
:10575000FF920F931F93CF93DF93EC01FC01E25B69
:10576000FF4F60817181828193810E94D4496B01D6
:105770007C016FA578A989A99AA90E94D6499B01A5
:10578000AC0160E074E284E799E40E945F424B015F
:105790005C01FE01E65AFF4F608171818281938135
:1057A0000E94D4499B01AC01C501B4010E945F4233
:1057B0004B015C018E010E5A1F4F20E030E040E0AB
:1057C0005FE30E94354A9B01AC01C701B6010E940C
:1057D000F4410E94D542F8016083718382839383F0
:1057E000CA5ADF4FA5019401C701B6010E94F441D6
:1057F0000E94D542688379838A839B83DF91CF910E
:105800001F910F91FF90EF90DF90CF90BF90AF90DE
:105810009F908F9008950F931F93CF93DF93FC0178
:10582000E859FF4F20812223C1F07A97008111812E
:1058300022813381389640815181628173810417BE
:1058400015072607370718F1EC010E948E0ACE01D2
:10585000DF91CF911F910F9174CFFC01E25AFF4F5E
:1058600020812223A1F07097008111812281338150
:105870003496408151816281738104171507260790
:10588000370728F0DF91CF911F910F91F1CEDF9173
:10589000CF911F910F9108952F923F924F925F9257
:1058A0006F927F928F929F92AF92BF92CF92DF9230
:1058B000EF92FF920F931F93CF93DF93CDB7DEB795
:1058C00062970FB6F894DEBF0FBECDBF8C017C018E
:1058D00025E4E20EF11CD7018C919801215A3F4F2B
:1058E000F801E05AFF4F6F01A801435C5F4F4A0186
:1058F00014971D01882341F0F80183A5D9018C93E9
:1059000081E0F60180832FC0DA014D915D916D91A8
:105910007C91F10180819181A281B381BB24B394F8
:10592000481759076A077B070CF0B12CF901B082C0
:1059300077FF07C070956095509541955F4F6F4F09
:105940007F4FB7FF07C0B095A095909581959F4F69
:10595000AF4FBF4F21E0481759076A077B070CF488
:1059600020E0D6012C93F401408151816281738142
:10597000411551056105710559F4F801838D948D28
:10598000A58DB68DE65AFF4F80839183A283B383A2
:10599000F10180819181A281B381F80141AC52ACC7
:1059A00063AC74AC9801225A3F4F5901481659060E
:1059B0006A067B0634F4481759076A077B077CF0B0
:1059C0000AC084159505A605B7052CF4841795071C
:1059D000A607B70724F0D7018C918823D9F0F501E9
:1059E00080818823B9F0D7018C91811105C0F7011E
:1059F000808181110FC006C060E0C80117DE8111EF
:105A0000F6CF17C0D6016C9181E06827C8010EDE81
:105A1000882379F0D5011C9260E0C80107DE882355
:105A200009F4C6C1F801FD96108211821282138218
:105A3000BFC1D80193962D913D914D915C91969760
:105A400029833A834B835C8357962D913D914D91E9
:105A50005C915A972D833E834F8358875B962D9197
:105A60003D914D915C915E9729873A874B875C8782
:105A7000F10180819181A281B381F801FD96C080FE
:105A8000D180E280F380F80141AD52AD63AD74ADD9
:105A9000EE59FF4F1082319610823801F4E66F0EF6
:105AA000711CF301108298012B593F4FF9011082AC
:105AB000329610824C015D01841A950AA60AB70A33
:105AC000B7FE08C0B094A09490948094811C911C5F
:105AD000A11CB11C481759076A077B072CF4C41A8C
:105AE000D50AE60AF70A04C0C81AD90AEA0AFB0A64
:105AF000D501C401B595A795979587958D879E8704
:105B0000AF87B88BD801A959BF4F1D01F7FC05C05D
:105B10008C149D04AE04BF044CF4F801078CF0A172
:105B2000E02DFA8BE98B81E0D9011BC02D853E85E4
:105B30004F8558892C153D054E055F0508F454C066
:105B400089819A81AB81BC818C159D05AE05BF050D
:105B500064F42D813E812F5F3F4F3A8B298B81E08A
:105B6000D3018C93F10180839EC0C701B6010E94CE
:105B7000D6492B013C0169817A818B819C810E94ED
:105B8000D6499B01AC01C301B2010E945F422B01C7
:105B90003C016D817E818F81988529853A854B8571
:105BA0005C85621B730B840B950B0E94D6499B018D
:105BB000AC01C301B2010E94354A2B013C01698549
:105BC0007A858B859C850E94D6499B01AC01C301D7
:105BD000B2010E94F4410E94CF427A8B698B81E02E
:105BE000F801EE59FF4F5CC0D501C40129813A810B
:105BF0004B815C81821B930BA40BB50BC816D90695
:105C0000EA06FB065CF42D813E812E5F3F4F3A8B06
:105C1000298B81E0F801EC59FF4F42C0C501B40166
:105C20006C197D098E099F090E94D6492B013C0100
:105C300069817A818B819C810E94D6499B01AC014C
:105C4000C301B2010E945F422B013C016D817E8144
:105C50008F81988529853A854B855C85621B730BFE
:105C6000840B950B0E94D6499B01AC01C301B20184
:105C70000E94354A2B013C0169857A858B859C857C
:105C80000E94D6499B01AC01C301B2010E94F441BC
:105C90000E94CF427A8B698B81E0F801ED59FF4F6A
:105CA0008083D1018C93F80184818823B1F00E9414
:105CB0006E08D80112964D905C901397052C000C3D
:105CC00066087708DC01CB0184199509A609B70994
:105CD000893E9340A105B10568F4F801E65AFF4FEB
:105CE00029893A89C901A0E0B0E080839183A28329
:105CF000B38392CE0E946E08D80113967C936E9364
:105D000012978AE494E00E94E5368DEF95E00E94B8
:105D1000E53660E070E0CB010E94313783E096E029
:105D20000E94E536C701B6010E94313789E096E04E
:105D30000E94E536C501B4010E9431378FE096E03C
:105D40000E94E5364AE06D857E858F8598890E94A0
:105D5000E63686E196E00E94E53669817A818B819C
:105D60009C810E9431378CE196E00E94E53669857E
:105D70007A858B859C850E94313782E296E00E946D
:105D8000E5366D817E818F8198850E94313788E26A
:105D900096E00E94E5368EE794E00E94E536898918
:105DA0009A890E94163886EC93E00E94E53695CFDA
:105DB00062960FB6F894DEBF0FBECDBFDF91CF91D4
:105DC0001F910F91FF90EF90DF90CF90BF90AF9019
:105DD0009F908F907F906F905F904F903F902F900B
:105DE00008950F931F93FC01EB5BFF4F208121115E
:105DF00010C038970081118122813381349640810F
:105E0000518162817381041715072607370744F40F
:105E100004C0FC0123A5222319F01F910F914DCB43
:105E20001F910F9130CBFC011382128214821682D3
:105E3000158210861782128611861486138616869E
:105E40001586108A1786128A118A148A138ADC0131
:105E5000A25ABF4F1C9211AE12AE13AE14AE919760
:105E60001D921D921D921C92139714961D921D92C5
:105E70001D921C92139714961C925A961C9211967E
:105E80001C9212961C9211961C9211961C921196BD
:105E90001C9211961C9211961C9211961C921196AE
:105EA0008BEE97E011969C938E93129611961C920E
:105EB0001E92129687EE97E011969C938E931296FF
:105EC00011961C921E92129683EE97E011969C9367
:105ED0008E93129611961C921E9212968FED97E059
:105EE0008D939C93E958FF4F1182108208950E9470
:105EF0001A220C9481220E941A220C944B21CF93D7
:105F0000DF93EC01FC01E655FD4F1082E558F109E5
:105F10008081811103C0CE014096E9DAFE01EA5D7D
:105F2000FD4F8081811104C0CE0187579F4FDFDA7A
:105F3000FE01E95DFD4F8081811104C0CE018E5FBD
:105F40009E4FD5DA64E670E080E090E0DF91CF917B
:105F50000C9436082F923F924F925F926F927F92ED
:105F60008F929F92AF92BF92CF92DF92EF92FF9269
:105F70000F931F93CF93DF93EC010E94EC0EFE0171
:105F8000E758FD4F809138089091390891838083BC
:105F90000E94EC0EFE01E558FD4F80913A08909169
:105FA0003B08918380830E94EC0EFE01E358FD4F75
:105FB00080913C0890913D08918380830E94EC0E73
:105FC0008E0101581D4F60914C0870914D08072EAD
:105FD000000C880B990B0E94D649F80160837183ED
:105FE000828393830E94EC0E1E01FDE72F1AFDEFC2
:105FF0003F0A60914E0870914F08072E000C880BE5
:10600000990B0E94D649F101608371838283938347
:106010000E94EC0E20E030E048EC52E4F801608190
:106020007181828193810E945F422B013C0120E0BB
:1060300030E048EC52E4F10160817181828193810A
:106040000E945F424B015C016091500870915108C1
:10605000072E000C880B990B0E94D64920E030E0F7
:1060600048EC52E40E945F426B017C012AE037ED6C
:1060700043E25CE3C301B2010E94014318168CF4B1
:1060800020E030E046EC52E4C301B2010E94D04966
:1060900087FD0FC0412C512C46EC642E42E4742E37
:1060A00008C05AE0452E57ED552E53E2652E5CE3AD
:1060B000752EF80140825182628273822AE037EDA8
:1060C00043E25CE3C501B4010E94014318168CF45D
:1060D00020E030E046EC52E4C501B4010E94D04912
:1060E00087FD0FC0812C912C26ECA22E22E4B22E2B
:1060F00008C03AE0832E37ED932E33E2A32E3CE323
:10610000B32EF10180829182A282B3822AE037ED20
:1061100043E25CE3C701B6010E94014318168CF408
:1061200020E030E046EC52E4C701B6010E94D049BD
:1061300087FD0FC0C12CD12C86ECE82E82E4F82E0E
:1061400008C09AE0C92E97EDD92E93E2E92E9CE380
:10615000F92EFE01E957FD4FC082D182E282F3821F
:106160000E94EC0E80912C0890912D08FE01E257C0
:10617000FD4F918380830E94EC0E80912E089091B8
:106180002F08FE01E057FD4F918380830E94EC0EA3
:106190008091300890913108FE01EE56FD4F9183B9
:1061A00080830E94EC0E8091400890914108FE018E
:1061B000EC56FD4F918380830E94EC0E8091420843
:1061C00090914308FE01EA56FD4F918380830E941F
:1061D000EC0E8091440890914508FE01E856FD4F71
:1061E000918380830E94EC0E809154089091550811
:1061F000FE01E656FD4F918380830E94EC0E809154
:10620000560890915708FE01E456FD4F9183808314
:106210000E94EC0E8091580890915908FE01E256B8
:10622000FD4F918380830E94EC0E809160089091D5
:106230006108FE01E056FD4F918380830E94EC0EC1
:106240008091620890916308FE01EE55FD4F9183A5
:1062500080830E94EC0E8091640890916508FE0195
:10626000EC55FD4F918380830E94EC0E80912408B1
:1062700090912508FE01E557FD4F019719F481E043
:10628000808301C010820E94EC0E809126089091BC
:106290002708FE01E457FD4F019719F481E0808340
:1062A00001C010820E94EC0E80912808909129086C
:1062B000C357DD4F019719F481E0888301C018822C
:1062C000DF91CF911F910F91FF90EF90DF90CF90D2
:1062D000BF90AF909F908F907F906F905F904F9006
:1062E0003F902F9008952F923F924F925F926F921E
:1062F0007F928F929F92AF92BF92CF92DF92EF9256
:10630000FF920F931F93CF93DF93CDB7DEB7AD9777
:106310000FB6F894DEBF0FBECDBF9DA78CA77A83C2
:1063200069830E94C8228CA59DA514DE8CA59DA51D
:10633000DEDD8CA59DA5DFDD29813A812130310587
:1063400009F43FC02230310509F473C0232B09F052
:10635000A8C02CA43DA430E1230E311C4CA55DA5A2
:1063600045585E4F58874F83ECA5FDA5EF5CFD4F68
:106370005081598B8CA59DA5815B9D4F9E878D87F4
:10638000ACA5BDA5A758BD4FBB8BAA8BECA5FDA5A1
:10639000E557FD4FFB8FEA8F2CA53DA526523E4FBA
:1063A000388B2F874CA55DA54D5B5D4F5D8F4C8F66
:1063B0008DE890E0998F888FA5E1B0E0BD8BAC8B24
:1063C00073C02CA43DA4B9E82B0E311CECA5FDA58F
:1063D000EB56FE4FF887EF83ECA5FDA5EE5CFD4F75
:1063E0002081298B4CA55DA54D5A5D4F5E874D8759
:1063F0008CA59DA585589D4F9B8B8A8BACA5BDA573
:10640000A457BD4FBB8FAA8FECA5FDA5E452FE4F4C
:10641000F88BEF872CA53DA5295B3D4F3D8F2C8F39
:106420004EE850E0598F488F86E190E09D8B8C8B31
:106430003BC02CA43DA49EEF291A390AACA5BDA5EA
:10644000A155BE4FB887AF83ECA5FDA5ED5CFD4F10
:10645000B081B98BECA5FDA5E95AFD4FFE87ED870C
:106460002CA53DA523583D4F3B8B2A8B4CA55DA504
:1064700043575D4F5B8F4A8F8CA59DA582529E4FDF
:10648000988B8F87ACA5BDA5A95BBD4FBD8FAC8F89
:10649000EFE8F0E0F98FE88F27E130E03D8B2C8BBF
:1064A00003C08EE296E00CC0C1010E94B40A8111C3
:1064B00005C0C1010E94A70A882331F085EF96E04C
:1064C00084D481E090E01EC48AE494E07ED481EA22
:1064D00096E07BD4D1018C91B9D48BE297E075D44E
:1064E00086EC93E072D481E090E0EF85F8899183A7
:1064F00080830CA51DA506521E4FD8014D915C91BD
:10650000B1018CA59DA50E942613C10104D8F101FB
:1065100083A59101215A3F4F3901882339F0C101E8
:106520000E945D2A81E0D3018C9305C0C1010E94C5
:10653000432AF30110828F8198850E94590A7101C4
:10654000FDE3EF0EF11CD7016D937D938D939C932A
:106550001397ED85FE851082118212821382ECA5BD
:10656000FDA5E15BFD4F1082118212821382ECA522
:10657000FDA5ED5AFD4F1082118212821382ECA507
:10658000FDA5E95AFD4F108211821282138286E026
:1065900090E0AF85B8898D939C93F801408151813B
:1065A000B1018CA59DA50E94261341E050E0B101E8
:1065B0008CA59DA50E940913412C512C32014394B6
:1065C00089819A8185579D4F2CA53DA5280F391F9C
:1065D0003F8F2E8F49815A81440F551F440F551FFD
:1065E0005C834B83CA0181589D4FACA5BDA5A80F04
:1065F000B91FB9A3A8A389819A81835B9E4F880F95
:10660000991FECA5FDA5E80FF91FFBA3EAA3CA019A
:1066100083599D4F2CA53DA5280F391F3DA32CA3C1
:106620000C974CA55DA5480F591F5FA34EA38B8106
:106630009C81815B9D4FACA5BDA5A80FB91FB9A7D3
:10664000A8A78B819C81ECA5FDA58E0F9F1F9C01A7
:1066500025503E4F3A872987FBA6EAA68E8C9F8C51
:10666000A8A0B9A0CAA0DBA0ECA0FDA00EA11FA10C
:1066700028A539A54F815885B1018CA59DA50E94FB
:10668000832984E09AE00E9422031816190624F058
:106690001E821D8210E010C084E09AE00E94000378
:1066A0008F7D85349105A1F785EE94E08ED341E08E
:1066B00050E05E834D8311E0C1010E94B40A811154
:1066C0001DC0C1010E94A70A811118C0111116C076
:1066D000AA89BB896D917C91072E000C880B990BC0
:1066E0000E94D6499B01AC01ED85FE8560817181D8
:1066F000828193810E94D04987FD6DC283ED96E02F
:1067000064D3C1010E94A70A811162C242E050E035
:10671000B1018CA59DA50E9409138AE494E055D38C
:1067200081EA96E052D3D1018C9190D388EA96E029
:106730004CD386EC93E049D3ED81FE81EF2BD1F46D
:106740008BEB96E042D38EE794E03FD38BEB94E063
:106750003CD38C899D896AD48EE794E036D38DEB47
:1067600094E033D3F9898F2F90E060D40E941A22ED
:106770000E9439218CA59DA5BADB8CA59DA5BBDB0C
:106780008AE494E022D381EA96E01FD3D1018C9170
:106790005DD38FEB96E019D386EC93E016D3ED85AD
:1067A000FE851082118212821382D1019B968C91F8
:1067B0008101015A1F4F882331F0C1010E94432AF1
:1067C000F801108206C0C1010E945D2A81E0D80153
:1067D0008C938F8198850E94590AF101FD96608300
:1067E000718382839383ECA5FDA5E15BFD4F10824D
:1067F000118212821382ECA5FDA5ED5AFD4F108285
:10680000118212821382ECA5FDA5E95AFD4F108278
:106810001182128213828F8198850E94590A6C8B93
:106820007D8B8E8B9F8B21E030E040E050E029870C
:106830003A874B875C8789819A8185579D4F4CA504
:106840005DA5480F591F5F8F4E8F8B819C818158AA
:106850009D4FACA5BDA5A80FB91FB9A3A8A3898159
:106860009A81835B9E4F880F991FECA5FDA5E80FC9
:10687000F91FFBA3EAA38B819C8183599D4F2CA513
:106880003DA5280F391F3DA32CA38B819C818F59D7
:106890009D4F4CA55DA5480F591F5FA34EA38B814B
:1068A0009C81815B9D4FACA5BDA5A80FB91FB9A761
:1068B000A8A749845A8491E0491A51083201AD8150
:1068C000BE81AB2B09F0B8C08E8C9F8CA8A0B9A05C
:1068D000CAA0DBA0ECA0FDA00EA11FA128A539A590
:1068E0004F815885B1018CA59DA50E94832984E024
:1068F0009AE00E9422031816190614F010E010C046
:1069000084E09AE00E9400038F7D85349105B1F701
:1069100085EE94E05AD2E1E0F0E0FE83ED8311E0F1
:10692000FAE04F16510438F4AD85BE851D921D92D4
:106930001D921C921397B989C101B111DEC10E9449
:10694000A70A811175C0112311F0320171C0EA89C3
:10695000FB8960817181072E000C880B990B0E94C6
:10696000D6499B01AC01AD85BE856D917D918D9120
:106970009C910E94D04987FFE8CFC1010E94382B2B
:106980006B807C80ECA5FDA56E0E7F1EF5E06F1A76
:10699000FEEF7F0AD3012D913D914D915C9160E511
:1069A00073EC80E090E00E94024BC9010E942B082A
:1069B000F3012081318142815381A3E0B0E00E9444
:1069C0001E4B9B01AC0169857A858B859C850E9455
:1069D000024B672B682B692B39F486E493E0F5D1E1
:1069E0000E941A220E943921C1010E948E0AEB8165
:1069F000FC812CA53DA5E20FF31FE550FE4F208141
:106A000031814281538160E573EC80E090E00E9427
:106A1000024BC9010E942B0889859A85AB85BC85EC
:106A20000196A11DB11D89879A87AB87BC8741CF8D
:106A300083ED96E0CAD104C0E1E0F0E0FE83ED838F
:106A40008AE494E0C2D181EA96E0BFD1D1018C9171
:106A5000FDD187EE96E0B9D186EC93E0B6D18F8177
:106A600098850E94590AEA8DFB8DEF2BA1F0DC017D
:106A7000CB012C893D894E895F89821B930BA40B26
:106A8000B50BB7FF07C0B095A095909581959F4F26
:106A9000AF4FBF4F3C014D815E81452B71F58BEBB4
:106AA00096E093D18EE794E090D18BEB94E08DD17A
:106AB000888D998DBBD28EE794E087D18DEB94E0E1
:106AC00084D1B301072C000C880B990B0E94D64986
:106AD0006B017C01AC8DBD8D6D917D918D919C91F3
:106AE0000E94D6499B01AC01C701B6010E945F42DA
:106AF000DFD10E941A220E94392185E090E0EF85C3
:106B0000F889918380830CA51DA506521E4FD801DC
:106B10004D915C91B1018CA59DA50E942613C101E8
:106B20000E94772A8CA59DA5E2D98CA59DA5E3D9C5
:106B3000E981FA81E130F105A1F0E230F10501F1DE
:106B4000EF2B61F50E941A22C301770CAA0BBB0B35
:106B50008093200990932109A0932209B0932309DF
:106B60001DC00E941A22C301770CAA0BBB0B809395
:106B7000240990932509A0932609B09327090EC0F4
:106B80000E941A22C301770CAA0BBB0B8093280921
:106B900090932909A0932A09B0932B090E941A22E5
:106BA0000E948C21AF85B8891D921C92F80140810A
:106BB0005181B1018CA59DA50E94261340E050E0B3
:106BC000B1018CA59DA50E9409138D819E819AC05B
:106BD00031E0398B9BCDC1010E94382BA985BA8544
:106BE0002D913D914D915C9160E573EC80E090E0DA
:106BF0000E94024BC9010E942B088201E985FA8597
:106C00002081318142815381A3E0B0E00E941E4B7C
:106C10009B01AC01C301B2010E94024B672B682BA0
:106C2000692B39F486E493E0D0D00E941A220E94A6
:106C30003921A985BA856D917D918D919C9126E030
:106C400030E040E050E00E94024BC301B2010E94DC
:106C5000024B672B682B692B79F58AE494E0B5D059
:106C60008DE596E0B2D0C801E1D18AE696E0ADD0DC
:106C7000ED85FE85608171818281938119D189E7DB
:106C800096E0A3D0AA89BB898D919C91CFD185E84C
:106C900096E09BD0EAA5FBA56081718182819381FA
:106CA000E0D083E996E091D08F8198850E94590ABF
:106CB000D8D086EC93E089D0C1010E948E0AA985C4
:106CC000BA852D913D914D915C9160E573EC80E02A
:106CD00090E00E94024BC9010E942B08BFEF4B1AA3
:106CE0005B0A6B0A7B0AED81FE81EF2B09F4B6CCBF
:106CF00021E030E03E832D8309CD0E94B40A81114A
:106D000024CE21CEAD960FB6F894DEBF0FBECDBF18
:106D1000DF91CF911F910F91FF90EF90DF90CF9077
:106D2000BF90AF909F908F907F906F905F904F90AB
:106D30003F902F900895CF93DF93FC01E353FE4FD4
:106D4000408151814115510559F1EC01CF52DE4F7F
:106D50002881398187539E4F24173507C8F4FC01D9
:106D600080819181009761F0FC01E20FF31F808127
:106D70008A3041F08D3029F486EC93E026D002C0B1
:106D800080E064D08881998101969983888308C0C6
:106D900040E050E068EC73E00E94260619821882F9
:106DA000DF91CF910895009769F0FC0101900020D8
:106DB000E9F73197AF01481B590BBC0184E09AE019
:106DC0000C94D50280E090E00895EDCF8F929F92D1
:106DD000AF92BF920F931F93CF93DF93CDB7DEB7E0
:106DE000A1970FB6F894DEBF0FBECDBF19A24230F7
:106DF00008F44AE08E010F5D1F4F842E912CA12CC8
:106E0000B12CA50194010E942E4BE62FB901CA01B5
:106E100001501109EA3014F4E05D01C0E95CD801C9
:106E2000EC93232B242B252B61F7C801BCDFA19603
:106E30000FB6F894DEBF0FBECDBFDF91CF911F918B
:106E40000F91BF90AF909F908F900895E091040AAA
:106E5000F091050A0190F081E02D682F84E09AE01E
:106E60001994CF92DF92EF92FF92CF93DF9397FF27
:106E700017C06B017C018DE2E9DFEC016627772703
:106E8000CB016C197D098E099F094AE09FDF8C0FA9
:106E90009D1FDF91CF91FF90EF90DF90CF900895ED
:106EA0004AE0DF91CF91FF90EF90DF90CF908ECFAF
:106EB0008F929F92AF92BF92CF92DF92EF92FF920A
:106EC000CF93DF936B017C019B01AC010E940543D2
:106ED000882319F08AE497E027C046015701E89417
:106EE000B7F82FEF3FEF4FE75FE7C501B4010E940E
:106EF000054381110DC02FEF3FEF4FE75FE7C5015D
:106F0000B4010E94D04918161CF48EE497E00CC01E
:106F10002FEF3FEF4FE75FE4C701B6010E94014347
:106F200018166CF482E597E0DF91CF91FF90EF9017
:106F3000DF90CF90BF90AF909F908F9034CF2FEF86
:106F40003FEF4FE75FECC701B6010E94D04987FDD4
:106F5000E9CF20E030E0A901C701B6010E94D04985
:106F600087FF08C08DE272DFEC01F7FAF094F7F8C2
:106F7000F09402C0C0E0D0E02AE037ED43EA5BE3E2
:106F8000C701B6010E94F4414B015C010E94D54249
:106F90006B017C010E94D4499B01AC01C501B40185
:106FA0000E94F3414B015C014AE0C701B6010EDFCC
:106FB000C80FD91F8EE24ADFC80FD91F20E030E08A
:106FC00040E251E4C501B4010E94354A4B015C0125
:106FD0000E94D5426B01E12CF12C4AE0C701B601B9
:106FE000F5DEC80FD91FC701B6010E94D4499B0125
:106FF000AC01C501B4010E94F34120E030E040E261
:1070000051E40E94354A0E94D54280E090E04AE077
:10701000DDDE8C0F9D1FDF91CF91FF90EF90DF9011
:10702000CF90BF90AF909F908F900895BC01990F23
:10703000880B990B16CF789484B5826084BD84B593
:10704000816084BD85B5826085BD85B5816085BD63
:1070500080916E00816080936E001092810080911B
:1070600081008260809381008091810081608093A3
:107070008100809180008160809380008091B100C8
:1070800084608093B1008091B00081608093B000F3
:107090008091910082608093910080919100816045
:1070A0008093910080919000816080939000809106
:1070B000A10082608093A1008091A10081608093F3
:1070C000A1008091A00081608093A00080912101A7
:1070D0008260809321018091210181608093210150
:1070E0008091200181608093200180917A008460EA
:1070F00080937A0080917A00826080937A008091F8
:107100007A00816080937A0080917A008068809311
:107110007A001092C10061E086E30E94EF0761E00F
:1071200087E30E94EF0761E086E20E94EF0761E0DB
:107130008AE10E94EF0761E08CE10E94EF0761E0C5
:1071400088E10E94EF0762E083E00E94EF0762E0BF
:1071500082E00E94EF0762E080E10E94EF0762E0B8
:1071600081E10E94EF0762E08FE10E94EF0762E099
:1071700081E20E94EF0761E08CE30E94EF0761E08B
:107180008DE30E94EF0761E088E30E94EF0762E071
:107190008EE00E94EF0762E08FE00E94EF0762E05E
:1071A00087E10E94EF0762E089E10E94EF0762E059
:1071B00083E20E94EF0762E085E20E94EF0761E050
:1071C0008EE20E94EF0761E080E30E94EF0761E03A
:1071D0008EE30E94EF0762E082E10E94EF0762E027
:1071E00083E10E94EF0762E08BE10E94EF0762E01B
:1071F0008DE10E94EF0762E087E20E94EF0762E004
:1072000089E20E94EF0761E08AE00E94EF0761E0F7
:1072100088E00E94EF0761E089E00E94EF0761E0EB
:107220008DE00E94EF0762E08FE30E94EF0762E0CB
:107230008BE30E94EF0762E088E20E94EF0762E0C2
:1072400080E40E94EF0762E08AE20E94EF0762E0BA
:107250008CE20E94EF0762E081E40E94EF0762E0A7
:1072600082E40E94EF0762E084E30E94EF0762E09D
:1072700085E30E94EF0762E080E00E94EF0762E092
:1072800081E00E94EF0762E089E30E94EF0762E07D
:107290008AE30E94EF0762E081E30E94EF0762E069
:1072A00082E30E94EF0762E083E30E94EF0762E05F
:1072B0008BE20E94EF0762E08DE20E94EF0762E03E
:1072C0008FE20E94EF0762E080E20E94EF0761E038
:1072D00086E20E94EB0661E088E10E94EB0661E035
:1072E00088E30E94EB0661E08EE30E94EB06E091EA
:1072F000140AF091150A82E08083E091100AF0915F
:10730000110A1082E091120AF091130AD0E1D083A1
:1073100010921C0AE091180AF091190A86E0808305
:10732000E091160AF091170A808180618083E091D4
:10733000160AF091170A808188608083E091160A0E
:10734000F091170A808180688083E091160AF0919D
:10735000170A80818F7D808364E670E080E090E092
:107360000E9436080E946D140E94E00F0E94B6141D
:107370000E94861482EE94E09093570780935607FC
:10738000C1E0C0936F00D093810010928000C09341
:107390002E0980E092E090932D0980932C09909320
:1073A00087008093860081E18093810010928100A4
:1073B000109285001092840080912E098061809344
:1073C00081000E946E086093CC097093CD09809370
:1073D000CE099093CF090E94EC0E80918207909184
:1073E00083070197E1F482E693E0EFDC0E946D14DD
:1073F000CF931F921F921F921F92812C912CA12C30
:10740000B12CC12CD12C760197018601B701A601C0
:107410000E94EB160F900F900F900F900F900E940C
:10742000EC0E80918007909181070197E9F48AE73B
:1074300093E0CBDC0E946D141F9221E02F931F92EA
:107440001F921F92812C912CA12CB12CC12CD12CDC
:10745000760197018601B701A6010E94EB160F90F5
:107460000F900F900F900F900E94EC0E80917E076E
:1074700090917F070197E9F482E993E0A6DC0E94EE
:107480006D141F921F9221E02F931F921F92812C47
:10749000912CA12CB12CC12CD12C76019701860105
:1074A000B701A6010E94EB160F900F900F900F905E
:1074B0000F908AEA93E089DC84E09AE00E9422033C
:1074C000892B09F482C50E946E086093CC097093E1
:1074D000CD098093CE099093CF0984E09AE00E9471
:1074E00000038093CB09982F9F7D953479F02091EC
:1074F000C9093091CA09F901E956F64F80832F5F17
:107500003F4F3093CA092093C90906C00E941A222E
:1075100021E0DC0116962C938091C9099091CA094B
:107520008133910564F02AE02093CB09FC01E956F0
:10753000F64F208301969093CA098093C9098091E0
:10754000CB092091C9093091CA098A3039F4C9019F
:107550000197A4E6B9E0E7E9F9E004C02233310578
:10756000B4F733C5AF0147595940481759071CF4C0
:1075700041914D93F7CFFC01EC59F64F1082223028
:1075800031050CF41EC58DE093E01FDC8EE794E01E
:107590001CDC89EC93E019DC84E699E016DC89ECCC
:1075A00093E013DC86EC93E010DC8AE390E00E9429
:1075B00029448C01FC0112821382148215821682E6
:1075C00017821086118612861386148615861686F3
:1075D0001786108A118A128A138A148A158A168AC3
:1075E000178A108E118E128E138E148E158E168E93
:1075F000178E10A211A212A213A214A215A216A2F3
:1076000017A210A611A612A613A614A615A616A6B2
:1076100017A610AA11AA12AA13AA14AA15AA16AA82
:1076200017AA10AE11AE6CE072E084E699E00E94F9
:107630005945EC01888186548230F0F00E94EC0EAE
:10764000A0906407B0906507F801C6A8D7A8E0AC81
:10765000F1AC0E941A22C0921C09D0921D09E0923E
:107660001E09F0921F09C0910002D0910102C230A0
:10767000D10508F4EEC1E4C16BEC73E0CE010E94C9
:10768000FA43892B09F4C9C06EEC73E0CE010E9465
:10769000FA43892B09F4C1C062ED73E0CE010E9468
:1076A000FA43892B09F4BCC065ED73E0CE010E945A
:1076B000FA43892B09F4B4C069ED73E0CE010E944E
:1076C000FA43892B09F4AFC06DED73E0CE010E943F
:1076D000FA43892B09F4A7C060EE73E0CE010E9443
:1076E000FA43892B09F4A2C064EE73E0CE010E9434
:1076F000FA43892B09F49DC068EE73E0CE010E9425
:10770000FA43892B09F498C06CEE73E0CE010E9415
:10771000FA43892B09F493C060EF73E0CE010E9415
:10772000FA43892B09F48EC064EF73E0CE010E9406
:10773000FA43892B09F489C068EF73E0CE010E94F7
:10774000FA43892B09F484C06CEF73E0CE010E94E8
:10775000FA43892B09F47FC060E074E0CE010E94F7
:10776000FA43892B09F47AC064E074E0CE010E94E8
:10777000FA43892B09F475C068E074E0CE010E94D9
:10778000FA43892B09F470C06CE074E0CE010E94CA
:10779000FA43892B09F46BC060E174E0CE010E94CA
:1077A000FA43892B09F466C064E174E0CE010E94BB
:1077B000FA43892B09F461C068E174E0CE010E94AC
:1077C000FA43892B09F45CC06CE174E0CE010E949D
:1077D000FA43892B09F457C060E274E0CE010E949D
:1077E000FA43892B09F452C064E274E0CE010E948E
:1077F000FA43892B09F44DC068E274E0CE01FAD750
:10780000892B09F449C06CE274E0CE01F3D7892BCF
:1078100009F445C08FEF9FEF44C080E090E041C085
:1078200081E090E03EC08DE690E03BC08FE690E0C6
:1078300038C080E790E035C081E790E032C082E751
:1078400090E02FC083E790E02CC084E790E029C04F
:1078500088E790E026C089E790E023C08AE790E0BF
:1078600020C083E890E01DC084E890E01AC08DE855
:1078700090E017C08EE890E014C08FE890E011C04F
:1078800080E990E00EC081EA90E00BC085EB90E0CB
:1078900008C086EB90E005C087EB90E002C088EB63
:1078A00090E09093010280930002209709F4C6CEE5
:1078B0008881883559F4CE0101960E945645D80139
:1078C00012966D937D938D939C931597888189353E
:1078D00049F4CE0101960E945645F80166837783EC
:1078E0008087918788818A3559F4CE0101960E945C
:1078F0005645D8011A966D937D938D939C931D9751
:107900008881813451F4CE0101960E94564547D6B4
:10791000F80166877787808B918B8881823461F448
:10792000CE0101960E9456453AD6D80152966D93E3
:107930007D938D939C9355978881833451F4CE0128
:1079400001960E9456452BD6F801668B778B808F67
:10795000918F8881833559F4CE0101960E94564556
:10796000D8015A966D937D938D939C935D978881F2
:10797000803551F4CE0101960E94564510D6F8018B
:10798000668F778F80A391A38881863561F4CE01BD
:1079900001960E94564503D6D80192966D937D9329
:1079A0008D939C9395978881873551F4CE010196EC
:1079B0000E945645F4D5F80166A377A380A791A746
:1079C0008881853461F4CE0101960E945645E7D541
:1079D000D8019A966D937D938D939C939D97888102
:1079E000843551F4CE0101960E945645D8D5F80150
:1079F00066A777A780AB91AB88818D3461F4CE0107
:107A000001960E945645CBD5D801D2966D937D93B1
:107A10008D939C93D5978881813551F4CE01019641
:107A20000E945645BCD5F80166AB77AB80AF91AFED
:107A300060E374E080E090E00E945945EC0135CFAE
:107A4000DD24D394CE018F569109069720F0D12CD6
:107A500002C0DD24D3940E941A22DC0116968C9178
:107A6000882381F0CD36D10509F424C4CE0188578E
:107A700091098330910548F1CD97039730F181E06A
:107A800093E097C20115110519F48DEF92E091C2B0
:107A9000CF3FBFEFDB07C9F32097D1F480912F09C7
:107AA00090913009892B61F482E090E0D2D625E1F3
:107AB00032E0FC01318320839093300980932F09B9
:107AC000E0902F09F090300953C001151105E9F23B
:107AD000CC31D105B9F48091310990913209892BCB
:107AE00061F482E090E0B5D62FE132E0DC012D9325
:107AF0003C939093320980933109E0903109F090E2
:107B000032096AC0CD36D105B9F48091330990911C
:107B10003409892B61F482E090E09BD629E232E0BF
:107B2000FC01318320839093340980933309E090E2
:107B30003309F090340950C0CF36D105B9F48091A3
:107B4000350990913609892B61F482E090E081D665
:107B500023E332E0DC012D933C939093360980932C
:107B60003509E0903509F090360950C0E12CF12C30
:107B7000C037D105B9F48091370990913809892B24
:107B800061F482E090E065D62DE332E0FC013183C0
:107B900020839093380980933709E0903709F0905B
:107BA000380968C0C137D105B9F48091390990917D
:107BB0003A09892B61F482E090E04BD627E432E069
:107BC000DC012D933C9390933A0980933909E0901E
:107BD0003909F0903A0968C0C237D105B9F48091EB
:107BE0003B0990913C09892B61F482E090E031D609
:107BF00021E532E0FC013183208390933C0980939E
:107C00003B09E0903B09F0903C0968C0C337D105BF
:107C1000B9F480913D0990913E09892B61F482E08D
:107C200090E017D62BE532E0DC012D933C93909346
:107C30003E0980933D09E0903D09F0903E0968C0FF
:107C4000C437D105B9F480913F0990914009892B3F
:107C500061F482E090E0FDD525E632E0FC0131835D
:107C600020839093400980933F09E0903F09F09072
:107C7000400968C0C837D105B9F480914109909195
:107C80004209892B61F482E090E0E3D52FE632E0EF
:107C9000DC012D933C939093420980934109E0903D
:107CA0004109F090420968C0C937D105B9F4809103
:107CB000430990914409892B61F482E090E0C9D591
:107CC00029E732E0FC0131832083909344098093BB
:107CD0004309E0904309F090440968C0CA37D105D0
:107CE000B9F48091450990914609892B61F482E0AD
:107CF00090E0AFD523E832E0DC012D933C939093E4
:107D0000460980934509E0904509F090460968C00E
:107D1000CD38D105B9F48091470990914809892B54
:107D200061F482E090E095D52DE832E0FC013183EA
:107D300020839093480980934709E0904709F09089
:107D4000480968C0CE38D105B9F4809149099091AD
:107D50004A09892B61F482E090E07BD527E932E083
:107D6000DC012D933C9390934A0980934909E0905C
:107D70004909F0904A0968C0CF38D105B9F480911B
:107D80004B0990914C09892B61F482E090E061D518
:107D900021EA32E0FC013183208390934C098093E7
:107DA0004B09E0904B09F0904C0968C0C039D105EF
:107DB000B9F480914D0990914E09892B61F482E0CC
:107DC00090E047D52BEA32E0DC012D933C93909371
:107DD0004E0980934D09E0904D09F0904E0968C01E
:107DE000C13AD105B9F480914F0990915009892B7E
:107DF00061F482E090E02DD525EB32E0FC01318387
:107E000020839093500980934F09E0904F09F090A0
:107E1000500967C0C53BD105B9F4809151099091D3
:107E20005209892B61F482E090E013D52FEB32E008
:107E3000DC012D933C939093520980935109E0907B
:107E40005109F09052094DC0C63BD105B9F480915B
:107E5000530990915409892B61F482E090E0F9D4A0
:107E600029EC32E0FC013183208390935409809304
:107E70005309E0905309F090540933C0C73BD10532
:107E8000B9F48091550990915609892B61F482E0EB
:107E900090E0DFD423ED32E0DC012D933C9390930E
:107EA000560980935509E0905509F090560919C07C
:107EB000C83BD105B1F48091570990915809892B9D
:107EC00061F482E090E0C5D427EE32E0FC0131831A
:107ED00020839093580980935709E0905709F090B8
:107EE0005809E114F10489F48DEF92E00E94E5361F
:107EF0000E941A220E94392184E394E00E94D33622
:107F000086EC93E00E94D3365AC089EF92E00E943B
:107F1000E5360E941A220E9439210E941A221092EC
:107F2000590710925807C0E0D0E02196C130D10522
:107F300041F085EF92E00E94E5360E941A220E94ED
:107F40003921D701ED91FC910480F581E02DB80134
:107F5000C70119950E941A228090580790905907DE
:107F6000209719F3CA15DB051CF481149104E9F676
:107F700084E09AE00E942203181619062CF484E08B
:107F80009AE00E940003F4CF892809F47DC1DD2026
:107F900009F47DC10E94EC0E809162079091630705
:107FA000019709F074C10E941A2221E0FC01268386
:107FB0006EC10E94E5360E941A220E943921C80132
:107FC000DDD41092CA091092C90980916309811108
:107FD00071C00E941A22DC0116968C91882309F444
:107FE00069C00E946D14EC01FC01E655FD4F108242
:107FF00040960E94772ACE0187579F4F0E94772A8A
:10800000CE018E5F9E4F0E94772A0E9436167C0119
:108010008C01075C1F4FC1E0D0E05801B8E3AB1AF8
:10802000B108F50180818823D9F08AE494E00E94A8
:10803000E5368EE494E00E94E536CE010E941638C3
:1080400086EC93E00E94E53660E08C2F0E94EB0600
:1080500040E050E0BE01C7010E94E214D5011C922D
:10806000F80180818823F9F08AE494E00E94E536E3
:1080700085E694E00E94E536CE010E94163886EC33
:1080800093E00E94E53661E08C2F0E94EF0760E0EC
:108090008C2F0E94EB0641E050E0BE01C7010E9418
:1080A000E214D8011C9221960F5F1F4FC533D105F2
:1080B00009F0B3CF0E941A22FC01868180936309E4
:1080C000C0916109D09162090E94EC0EDC01129608
:1080D0008D919C911397C817D90789F00E94EC0ED7
:1080E000FC018281938190936209809361090E94CF
:1080F0006D140E94E00F0E94B6140E9486140E9424
:108100006E0860935D0970935E0980935F09909398
:1081100060090091CC091091CD092091CE093091D0
:10812000CF09601771078207930708F4A0C0DC012C
:10813000CB01801B910BA20BB30B89389341A10596
:10814000B10508F49EC00E941A22DC0116968C919B
:10815000882319F089E093E002C085E093E00E9453
:10816000E5360E941A220E9439210E946D14EC010A
:10817000FC01E557FD4F8081882341F0CE018558F1
:108180009E4F0E94590A4B015C0107C0FE01E35B50
:10819000FF4F80809180A280B3800E941A2280923B
:1081A000200990922109A0922209B0922309FE0190
:1081B000E457FD4F8081882341F0CE018B569E4FBE
:1081C0000E94590A4B015C0107C0FE01EA53FF4FB0
:1081D00080809180A280B3800E941A22809224091C
:1081E00090922509A0922609B0922709FE01E35733
:1081F000FD4F8081882341F0CE0181559E4F0E9422
:10820000590A4B015C0106C0C15CDE4F8880998031
:10821000AA80BB800E941A22809228099092290984
:10822000A0922A09B0922B090E941A220E948C2146
:108230000E946D140E94B7130E941A220E9481228C
:108240000E941A220E944B218091590990915A094B
:10825000A0915B09B0915C090196A11DB11D8093AD
:10826000590990935A09A0935B09B0935C090E9445
:108270006E086093CC097093CD098093CE099093DA
:10828000CF090E94BF0318C981EF92E002C08DEEB2
:1082900092E00E94E5360E941A220E9439210E9433
:1082A0001A2210921C0910921D0910921E09109298
:1082B0001F0985CE0115110509F027CCE6CB809169
:1082C000A10A9091A20A5AC31092070A1092060AB4
:1082D00088EE93E0A0E0B0E08093080A9093090A4A
:1082E000A0930A0AB0930B0A8EE493E09093050AD8
:1082F0008093040A85EC90E09093110A8093100A11
:1083000084EC90E09093130A8093120A80EC90E042
:108310009093150A8093140A81EC90E09093170AC9
:108320008093160A82EC90E09093190A8093180AC1
:1083300086EC90E090931B0A80931A0A10921D0A13
:1083400010921E0A10921F0A1092200A82E090E0FA
:1083500080D22EE533E0FC01318320839093A80A7C
:108360008093A70A68EC73E081EA9AE00E945006C5
:108370008091390B803320F09FEF90933A0B11C01E
:1083800080933A0B282F30E0F901EE0FFF1F2E0FDC
:108390003F1FF901E755F54F28EB3BE0328321837E
:1083A0008F5F803390F480933D0B282F30E0F901EC
:1083B000EE0FFF1F2E0F3F1FF901E755F54F28EB7A
:1083C0003BE0328321838F5F03C09FEF90933D0B8F
:1083D0008093390B0895EE0FFF1F881F8BBF079006
:1083E000F691E02D19945058BB27AA2713D00C946E
:1083F000B24A0E94A44A38F00E94AB4A20F039F4F5
:108400009F3F19F426F40C94A14A0EF4E095E7FB83
:108410000C949B4AE92F0E94C34A58F3BA1762078B
:1084200073078407950720F079F4A6F50C94E54AC4
:108430000EF4E0950B2EBA2FA02D0B01B90190017F
:108440000C01CA01A0011124FF27591B99F0593FC3
:1084500050F4503E68F11A16F040A22F232F342F0B
:108460004427585FF3CF469537952795A795F04059
:108470005395C9F77EF41F16BA0B620B730B840B6E
:10848000BAF09150A1F0FF0FBB1F661F771F881F26
:10849000C2F70EC0BA0F621F731F841F48F487957E
:1084A00077956795B795F7959E3F08F0B0CF939570
:1084B000880F08F09927EE0F97958795089512D0A9
:1084C0000C94B24A0E94AB4A58F00E94A44A40F071
:1084D00029F45F3F29F00C949B4A51110C94E64A11
:1084E0000C94A14A0E94C34A68F39923B1F355231F
:1084F00091F3951B550BBB27AA27621773078407B7
:1085000038F09F5F5F4F220F331F441FAA1FA9F34C
:1085100034D00E2E3AF0E0E831D091505040E6953C
:10852000001CCAF72AD0FE2F28D0660F771F881F9D
:10853000BB1F261737074807AB07B0E809F0BB0B8E
:10854000802DBF01FF2793585F4F32F09E3F5105AA
:1085500070F0F1C70C94E64A5F3FE4F3983ED4F321
:10856000869577956795B795F7959F5FC9F7880FBB
:10857000911D9695879597F90895E1E0660F771F0D
:10858000881FBB1F621773078407BA0720F0621B9E
:10859000730B840BBA0BEE1F88F7E095089505D096
:1085A0006894B1110C94E64A0895F5D788F09F5766
:1085B00090F0B92F9927B751A0F0D1F0660F771F2F
:1085C000881F991F1AF0BA95C9F712C0B13081F00F
:1085D000FCD7B1E00895F9C7672F782F8827B85FD7
:1085E00039F0B93FCCF3869577956795B395D9F770
:1085F0003EF490958095709561957F4F8F4F9F4F7A
:1086000008950FD708F48FEF08950BD7880B990BB7
:1086100008956F927F928F929F92AF92BF92CF9266
:10862000DF92EF92FF920F931F93CF93DF93EC01B2
:10863000009781F4CB01DF91CF911F910F91FF90B3
:10864000EF90DF90CF90BF90AF909F908F907F90F2
:108650006F90FFC0FC01E60FF71F9C01225031090B
:10866000E217F30708F4A8C0D9010D911C911197E6
:1086700006171707A8F00530110508F49BC0C801BC
:1086800004978617970708F495C002501109061B36
:10869000170B019311936D937C93CF016FD18AC017
:1086A0005B01A01AB10A4C01800E911EA091440BEF
:1086B000B091450B40E050E0E12CF12C109709F40B
:1086C0004AC0A815B905D1F56D907C90119763014A
:1086D00082E0C80ED11CCA14DB0480F1A3014A1940
:1086E0005B096A0182E0C80ED11C1296BC901297F9
:1086F0001396AC91B5E0CB16D10440F0B282A383BF
:1087000051834083D9016D937C930AC00E5F1F4F44
:10871000C301800F911FF90191838083EB2DFA2F04
:10872000E114F10431F0D7011396FC93EE93129704
:1087300041C0F093450BE093440B3CC08D919C915C
:1087400011974817590708F4AC017D0112960D9056
:10875000BC91A02DB3CF8091420B9091430B881513
:108760009905E1F446175707C8F4809102029091E9
:108770000302009741F48DB79EB7409106025091D5
:108780000702841B950BE817F907B0F4F093430B2D
:10879000E093420BF901718360830CC0CB0159D087
:1087A0007C01009749F0A801BE011BD0CE01E6D0A4
:1087B000C70104C0CE0102C080E090E0DF91CF91FC
:1087C0001F910F91FF90EF90DF90CF90BF90AF90EF
:1087D0009F908F907F906F90089581E090E0F89443
:1087E0006EC7FB01DC0102C001900D924150504068
:1087F000D8F70895FB01DC018D91019080190110DB
:10880000D9F3990B0895FB01DC0101900D92002032
:10881000E1F70895EF920F931F93CF93DF93E80151
:1088200047FD02C034E001C034E1E42F440FFF0BE8
:10883000F7FF03C0F195E195F109E32E022F2E2FEA
:10884000AE01B3D1CE01DF91CF911F910F91EF9087
:108850000895CF93DF938230910510F482E090E089
:10886000E091440BF091450B20E030E0C0E0D0E017
:10887000309711F14081518148175907C0F04817CE
:10888000590761F482819381209719F09B838A8331
:108890002BC09093450B8093440B26C021153105C6
:1088A00019F04217530718F49A01BE01DF01EF01D6
:1088B0000280F381E02DDCCF2115310509F1281B61
:1088C000390B2430310590F412968D919C911397B9
:1088D0006115710521F0FB019383828304C090939D
:1088E000450B8093440BFD01329644C0FD01E20F1D
:1088F000F31F81939193225031092D933C933AC0F9
:108900002091420B3091430B232B41F42091040220
:10891000309105023093430B2093420B20910202C9
:10892000309103022115310541F42DB73EB7409136
:10893000060250910702241B350BE091420BF09187
:10894000430BE217F307A0F42E1B3F0B2817390740
:1089500078F0AC014E5F5F4F2417350748F04E0F9B
:108960005F1F5093430B4093420B8193919302C03E
:10897000E0E0F0E0CF01DF91CF9108950F931F93D6
:10898000CF93DF93009709F48CC0FC0132971382D8
:1089900012820091440B1091450B0115110581F4D1
:1089A00020813181820F931F2091420B3091430B24
:1089B0002817390779F5F093430BE093420B71C008
:1089C000D80140E050E0AE17BF0750F412962D9149
:1089D0003C911397AD012115310509F1D901F3CF70
:1089E0009D01DA013383228360817181860F971F95
:1089F0008217930769F4EC0128813981260F371F0C
:108A00002E5F3F4F318320838A819B8193838283B2
:108A1000452B29F4F093450BE093440B42C0139689
:108A2000FC93EE931297ED01499159919E01240F09
:108A3000351FE217F30771F480819181840F951F30
:108A4000029611969C938E938281938113969C93A8
:108A50008E931297E0E0F0E0D80112968D919C91F0
:108A60001397009719F0F8018C01F6CF8D919C9126
:108A700098012E5F3F4F820F931F2091420B309140
:108A8000430B2817390769F4309729F41092450BE6
:108A90001092440B02C0138212821093430B009376
:108AA000420BDF91CF911F910F9108956627772791
:108AB00009C240E45BE000C0FA01A191B0810097D7
:108AC00019F41097E1F0CD01DC01CD010D900020EB
:108AD00011F4C00113C0FB012191222319F02015CC
:108AE000D9F7F3CFFB012191201519F41E921196AD
:108AF00006C02223C1F70D900020A1F7D001FA0192
:108B0000A193B0830895BB274A3031F4992322F40E
:108B1000BDE2909581959F4F30C0BB272A3051F41C
:108B2000992342F4BDE290958095709561957F4FB1
:108B30008F4F9F4F01C0BB27FA01A62F6217710507
:108B400081059105330B30FB66F0AA27660F771F6E
:108B5000881F991FAA1FA21710F0A21B63953850F7
:108B6000A9F7A05DAA3308F0A95DA19336F7B1116A
:108B7000B1931082CA0104C4BB27FB015527AA2761
:108B8000880F991FAA1FA41710F0A41B839550519A
:108B9000B9F7A05DAA3308F0A95DA193009779F712
:108BA000B111B1931192CB01EBC34F925F926F92CF
:108BB0007F929F92AF92BF92CF92DF92EF92FF92FD
:108BC0000F931F93CF93DF93CDB7DEB729970FB6DF
:108BD000F894DEBF0FBECDBF6A01122FB02E2BE37B
:108BE000201720F0FF24F394F00E02C0BCE3FB2E0C
:108BF0000F2D27E0AE014F5F5F4FCAD2AC018981D4
:108C0000982F9970913031F0E1FC06C0E0FE06C06B
:108C100090E205C09DE203C09BE201C090E0EE2D12
:108C2000E07183FF3CC0911102C083E001C084E089
:108C3000811718F4212F281B01C020E0E1110BC07F
:108C4000F601822F30E2882319F031938150FBCF57
:108C5000C20ED11C20E0992329F0D6019C93F60185
:108C600031966F01C6010396E2FE0AC03EE4D601CA
:108C70003C9341E411964C93119712963C9306C095
:108C80003EE6F601308341E641833283FC01322F18
:108C900040E2332309F442C041933150FACF82FFBE
:108CA00044C0911102C083E001C084E0811718F430
:108CB000212F281B01C020E0E1110BC0F601822FFB
:108CC00030E2882319F031938150FBCFC20ED11CC2
:108CD00020E0992329F0D6019C93F60131966F018B
:108CE000C6010396E2FE0BC039E4D6013C933EE494
:108CF00011963C93119736E412963C9307C039E6DF
:108D0000F60130833EE6318336E63283FC01322FB2
:108D100040E2332319F041933150FBCFFC01E20FC5
:108D2000F11D10828EEF9FEFB7C0F1E0911101C0ED
:108D3000F0E06F2F70E01416150624F49A012F5FEF
:108D40003F4F02C021E030E0260F371FBB2029F043
:108D50006B2D70E06F5F7F4F02C060E070E0260F08
:108D6000371F612F70E0261737071CF4121B212FC5
:108D700001C020E03E2D387159F4D601322F60E257
:108D8000332319F06D933150FBCFC20ED11C20E07C
:108D9000FF2331F0D6019C93B6016F5F7F4F6B01CB
:108DA000E1110BC0F601922F30E3992319F03193B2
:108DB0009150FBCFC20ED11C20E09F2D940F3A8121
:108DC000782F7071A72E84FF03C0313309F49150BE
:108DD000191624F4993018F098E001C091E0E42FBE
:108DE000852F57FF02C0E0E080E06E2F782FE0E093
:108DF000F0E0AEE29A2E3A01691A71082A01461A89
:108E0000570A0B2D10E01195019511096F3F8FEF57
:108E1000780729F4D6019C92C60101966C01461789
:108E2000570784F0661677066CF47F01E40CF51C96
:108E3000A1E0B0E0AC0FBD1FEA0EFB1ED7011196FA
:108E4000BC9002C090E3B92E615071093196C60101
:108E500001967C016017710724F0D601BC926C0169
:108E6000D5CF6417750741F4363320F4353321F438
:108E7000A11002C081E3B82EF601B082F701822F63
:108E800090E2882319F091938150FBCFF701E20F14
:108E9000F11D108280E090E029960FB6F894DEBFB5
:108EA0000FBECDBFDF91CF911F910F91FF90EF903B
:108EB000DF90CF90BF90AF909F907F906F905F902A
:108EC0004F9008956F927F928F929F92AF92BF9230
:108ED000CF92DF92EF92FF920F931F93CF93DF9386
:108EE000EC017B016115710519F0DB018D939C93F9
:108EF0008E010F5F1F4F7880872D90E021D2892B44
:108F000011F0E801F5CFBDE27B1205C00F5F1F4FE6
:108F10007980C1E008C0EBE27E1204C08E010E5FD2
:108F20001F4F7980C0E06801F1E0CF1AD10843E01B
:108F300050E064E174E0C6010BD2892BE9F46801CA
:108F400022E0C20ED11C45E050E06FE074E0C601A3
:108F5000FFD1892B21F4680187E0C80ED11CE114F0
:108F6000F10419F0D701CD92DC92C111F9C060E093
:108F700070E080E89FE7FDC043E050E06CE074E003
:108F8000C601E6D1892B51F4E114F10409F4EDC0D6
:108F90000E5F1F4FF70111830083E7C0680160E097
:108FA00070E0CB0100E010E0F601D0EDD70DDA3033
:108FB00050F52C2F2260622E2C2F2870C2FF05C086
:108FC000211127C00F5F1F4F24C0222311F0015031
:108FD0001109A5E0B0E09B01AC0130D34B015C016D
:108FE000880C991CAA1CBB1CC501B4016D0F711D16
:108FF000811D911D6839A9E97A078A07A9E19A07B5
:1090000040F0C66005C0DE3F51F4C3FD44C0C860F7
:109010006C2EBFEFCB1ADB0A7080C62DC5CF2D2F6B
:109020002F7D2531C1F540814D3211F4C06106C05C
:109030004B3221F0319621E030E006C03296D60165
:1090400011964C9122E030E0A0EDA40FAA3018F068
:10905000E21BF30B20C040E050E04038BCE05B076F
:109060005CF49A01220F331F220F331F420F531F4C
:10907000440F551F4A0F511D3196DF0111972C9156
:10908000A0EDA20FAA3048F3C4FF03C0519541954B
:109090005109040F151FC1FF07C0E114F10421F0AD
:1090A0003197D701ED93FC937FD1C370C33019F092
:1090B0006B017C0106C06B017C01F7FAF094F7F8B4
:1090C000F09420E030E0A901C701B60169D18823FE
:1090D00009F443C017FF06C0119501951109CBE2B1
:1090E000D4E002C0C3E4D4E05E01B8E1AB1AB10839
:1090F0004601BE2DAF2D90E2E92EF12C0E151F0575
:109100007CF0FE012591359145915491B4018B2F4E
:109110009A2FABD14B01B82FA92F0E191F09EECFF3
:109120002497F594E794CA15DB0541F76401EB2E0B
:10913000FA2E8E2D880F8F2D881F8F3F41F020E053
:1091400030E0A901C701B6012BD1811106C082E22E
:1091500090E09093470B8093460BC701B60109C07E
:1091600060E070E080E89FEF04C060E070E080ECB9
:109170009FE7DF91CF911F910F91FF90EF90DF90CC
:10918000CF90BF90AF909F908F907F906F900895F9
:10919000283008F027E03327DA01990F311D87FDC9
:1091A000916000966105710539F432602E5F3D9340
:1091B00030E32A95E1F708959F3F30F0803871053C
:1091C000610509F03C5F3C5F3D93913008F0806899
:1091D000911DDF93CF931F930F93FF92EF92192F5F
:1091E000987F9695E92F96959695E90FFF27EF556D
:1091F000FB4F99273327EE24FF24A701E7010590B1
:109200000894079428F4360FE71EF81E491F511DD5
:10921000660F771F881F991F0694A1F70590079482
:1092200028F4E70EF81E491F561FC11D770F881F2F
:10923000991F661F0694A1F70590079428F4F80E6D
:10924000491F561FC71FD11D880F991F661F771F03
:109250000694A1F70590079420F4490F561FC71FE5
:10926000D81F990F661F771F881F0694A9F784914E
:109270001095177041F0D695C79557954795F79477
:10928000E7941A95C1F7E7E4F4E068941590159116
:1092900035916591959105907FE27395E118F10AFA
:1092A000430B560BC90BD009C0F7E10CF11E431F4D
:1092B000561FC91FD01D7EF4703311F48A95E6CF76
:1092C000E894015030F0080F0AF40027021708F460
:1092D000202F2395022F7A3328F079E37D932A9566
:1092E000E9F710C07D932A9589F6069497956795BE
:1092F000379517951794E118F10A430B560BC90BD4
:10930000D00998F023957E9173957A3308F070E335
:109310007C932013B8F77E9170617D9330F0839534
:1093200071E37D9370E32A95E1F71124EF90FF90AC
:109330000F911F91CF91DF91992787FD9095089507
:109340009111F6C0803219F089508550D0F70895F8
:10935000FB01DC014150504088F08D9181341CF0BC
:109360008B350CF4805E659161341CF06B350CF428
:10937000605E861B611171F3990B0895881BFCCF09
:10938000DC01FC01672F71917723E1F7329704C06C
:109390007C916D9370836291AE17BF07C8F30895F7
:1093A00040D008F481E00895E89409C097FB3EF4AA
:1093B00090958095709561957F4F8F4F9F4F992322
:1093C000A9F0F92F96E9BB279395F69587957795A0
:1093D0006795B795F111F8CFFAF4BB0F11F460FF60
:1093E0001BC06F5F7F4F8F4F9F4F16C0882311F0B8
:1093F00096E911C0772321F09EE8872F762F05C0CC
:10940000662371F096E8862F70E060E02AF09A9566
:10941000660F771F881FDAF7880F9695879597F95B
:109420000895990F0008550FAA0BE0E8FEEF1616F5
:109430001706E807F907C0F012161306E407F50748
:1094400098F0621B730B840B950B39F40A2661F0BC
:10945000232B242B252B21F408950A2609F4A1405F
:10946000A6958FEF811D811D08950BD07BC06CD018
:1094700028F071D018F0952309F05DC062C0112466
:10948000A5C081D0A0F3959FD1F3950F50E0551F53
:10949000629FF001729FBB27F00DB11D639FAA2749
:1094A000F00DB11DAA1F649F6627B00DA11D661F98
:1094B000829F2227B00DA11D621F739FB00DA11DB9
:1094C000621F839FA00D611D221F749F3327A00D73
:1094D000611D231F849F600D211D822F762F6A2F0F
:1094E00011249F5750408AF0E1F088234AF0EE0F94
:1094F000FF1FBB1F661F771F881F91505040A9F7A1
:109500009E3F510570F017C061C05F3FECF3983E7D
:10951000DCF3869577956795B795F795E7959F5F07
:10952000C1F7FE2B880F911D9695879597F90895A1
:1095300099278827089597F99F6780E870E060E091
:1095400008959FEF80EC089500240A9416161706DC
:1095500018060906089500240A9412161306140624
:1095600005060895092E0394000C11F4882352F087
:10957000BB0F40F4BF2B11F460FF04C06F5F7F4F3F
:109580008F4F9F4F089557FD9058440F551F59F026
:109590005F3F71F04795880F97FB991F61F09F3FE0
:1095A00079F087950895121613061406551FF2CF09
:1095B0004695F1DF08C0161617061806991FF1CF59
:1095C00086957105610508940895E894BB27662780
:1095D0007727CB0197F90895F999FECF92BD81BD08
:1095E000F89A992780B50895262FF999FECF1FBACA
:1095F00092BD81BD20BD0FB6F894FA9AF99A0FBEBC
:1096000001960895052E97FB16F400940FD057FD90
:1096100005D024D007FC02D046F408C050954095F0
:10962000309521953F4F4F4F5F4F0895909580950E
:10963000709561957F4F8F4F9F4F089531D0A59FB3
:10964000900DB49F900DA49F800D911D112408953D
:10965000B7FFF4CFF3DF821B930B0895A1E21A2E1C
:10966000AA1BBB1BFD010DC0AA1FBB1FEE1FFF1FC6
:10967000A217B307E407F50720F0A21BB30BE40B16
:10968000F50B661F771F881F991F1A9469F760955D
:109690007095809590959B01AC01BD01CF01089517
:1096A000A29FB001B39FC001A39F700D811D112423
:1096B000911DB29F700D811D1124911D089512E01E
:1096C000C2EAD2E000E006C0802FFE010E94EB411A
:1096D0002196011DC33AD10780E00807A9F7F89445
:0296E000FFCFBA
:1096E200FFFF0000480B800001000000200A0D006F
:1096F2000000000000950FF20C430D0000000094E2
:109702000FF00C020D00000000F220141F7B22005B
:10971200000000F120121FB62000000000F020100F
:109722001F852000000000EF200E1F5420000000C3
:1097320000EE200C1F1B2000000000ED200A1FE29B
:109742001F00000000EC20081FA91F00000000EB12
:1097520020FE1E572200000000EA20061F521F00B2
:10976200000000E920041F611F00000000E8200241
:109772001F2C1F00000000E720001F161F00000022
:10978200009C0F000DE71E000000009B0FFE0C5C0A
:109792000E000000009A0FFC0C300E000000009931
:1097A2000FFA0C050E00000000980FF80CFE0D00D9
:1097B200000000970FF60CDD0C00000000930FEE86
:1097C2000CDA0C00000000960FF40C980D523033A6
:1097D20000523032005230370052303100523039AC
:1097E2000052383700523030005238370052303889
:1097F20000352E302E372E520000010000000100ED
:109802000000010000005238350052383400523056
:10981200350052303600523133005231320052316B
:109822003100523837005230340000000000580333
:10983200D5022203000314039E0300000000920FCE
:10984200EC0C52393920484F4D45205A204F4E20BA
:10985200535441525455500D0A0052393920484F41
:109862004D452059204F4E20535441525455500DCE
:109872000A0052393920484F4D452058204F4E207A
:10988200535441525455500D0A0052393920415215
:109892004455494E4F205354415254555020434F42
:1098A2004D504C4554450D0A002A004730004730C0
:1098B2003000473100473031004630390046390028
:1098C20046313100463132004631330046313400F0
:1098D20046313500463136004632300046323100DC
:1098E20046323200463331004633320046343100CC
:1098F20046343200463433004634340046363100B2
:109902004638310046383200463833004638340093
:10991200200A0D005239392068616E646C6572202C
:109922003D3D204E554C4C0D0A00523939002072F3
:109932006573657474696E67206469676974616CC4
:109942002070696E0020726573657474696E672099
:10995200616E616C6F672070696E0052383320004F
:109962005239392057696C6C207A65726F20580021
:109972005239392057696C6C207A65726F20590010
:109982005239392057696C6C207A65726F205A00FF
:10999200686F6D650D0A0052323100500056005258
:1099A2003939204572726F723A20696E76616C693C
:1099B2006420706172616D657465722069640D0A5C
:1099C200005234310052393920656D657267656E17
:1099D20063792073746F700D0A00523939206572F1
:1099E200726F720D0A005238320052393920737484
:1099F2006F707065640D0A00523939206572726F9A
:109A02007220002064656163746976617465206DFB
:109A12006F746F7220582064756520746F206D69B1
:109A22007373656420737465707300206465616389
:109A3200746976617465206D6F746F722059206449
:109A4200756520746F206D69737365642073746526
:109A52007073002064656163746976617465206D5A
:109A62006F746F72205A2064756520746F206D695F
:109A7200737365642073746570730052393920748E
:109A8200696D656F7574205820617869730D0A00DD
:109A92005239392074696D656F7574205920617867
:109AA20069730D0A005239392074696D656F7574D6
:109AB200205A20617869730D0A0020510052383112
:109AC20000205841002058420020594100205942AC
:109AD20000205A4100205A42005232300020737452
:109AE20061200020637572200020656E64200020D2
:109AF20068616C662000206C656E2000206D696EC6
:109B02002000206D6178200020737064200052399B
:109B1200392043616C6962726174696F6E2065728B
:109B2200726F723A20696E76616C6964206178693D
:109B3200732073656C65637465640D0A0020737429
:109B4200657020636F756E742000206D6973736594
:109B5200642073746570732000206D6178207374C3
:109B620065707320002063757220706F73206D74AE
:109B72007220002063757220706F7320656E6320FF
:109B8200002061786973200020617420737461720F
:109B920074696E6720706F696E74005232330020F0
:109BA20063616C6962726174696E67206C656E676D
:109BB200746800523939206D6F76656D656E742058
:109BC200646F6E650D0A0020617420656E642070FA
:109BD2006F696E74005239392043616C6962726137
:109BE20074696F6E206572726F723A20656E6420BE
:109BF20073746F7020616374697665206265666F45
:109C020072652073746172740D0A00206D6F76653F
:109C120020746F20737461727420666F72206361A6
:109C22006C6962726174696F6E006E616E00696E5A
:069C320066006F7666007B
:00000001FF
